:020000040800F2
:10500000001C0020D5500008C1880008C17F00089E
:105010000000000000000000000000000000000090
:1050200000000000000000000000000011970008D0
:105030000000000000000000919000084D9800085A
:10504000E7500008E7500008E7500008E750000864
:10505000E75000084D5D0008E7500008E7500008E1
:1050600000000000E7500008755C0008E7500008E9
:10507000E75000083185000800000000E7500008F4
:1050800000000000E75000080000000000000000E1
:10509000E750000800000000E7500008E750000853
:1050A000E7500008E7500008E750000819A1000881
:1050B000E7500008E7500008000000000000000072
:1050C0000348854600F0E8FC004800478DB400081E
:1050D000001C00200448804704480047FEE7FEE724
:1050E000FEE7FEE7FEE7FEE7E9980008C15000088A
:1050F00030B50B46014600202022012409E00D4670
:10510000D5409D4205D31D469540491B25469540F7
:1051100040191546521E002DF1DC30BDF0B51FB40C
:105120000646002082B005464024019100901BE015
:10513000019922460F46304600F098FB049A059BE1
:10514000801A994110D310461946224600F07EFB82
:10515000361A8F410197224601200021009F00F05E
:1051600075FB38184D4100902046641E0028DFDC96
:10517000019B00982946324607B0F0BD03460B4319
:105180009B0703D009E008C9121F08C0042AFAD2FD
:1051900003E00B780370401C491C521EF9D2704783
:1051A000D2B201E00270401C491EFBD270470022BF
:1051B000F6E710B513460A4604461946FFF7F0FF16
:1051C000204610BD30B504460020034600E05B1CBD
:1051D000934203D2E05CCD5C401BF8D030BDF8B503
:1051E00002464A40D40F42004B0052085B089A42E4
:1051F00002D20246084611464A0023D0C30D4A0097
:10520000DDB2120EAD1A202D35DA49020126490A07
:10521000F6058A19002C00D0524220214F1B11465E
:10522000B9402A411018C20D9A4221D0002C17D043
:10523000012D08DCDA05801AD20F8019D207DBB203
:1052400000F040FBF8BDDA05801A012340001B0680
:10525000C01880185A428018CA0F1043490007E04E
:105260004908C2071143DA05801A801940088018DE
:1052700000F020FBF8BD61000122511A001BF7E786
:105280000122D2075140AAE70122D2075040A6E7E7
:1052900070B502464A40D50F40004A00ED0740086D
:1052A0005208002814D0002A12D0C40DD30D410298
:1052B0000120C0055202490A520AE41A09181218BC
:1052C0007D34914201D3641C00E04900002C01DAD6
:1052D000002070BD0023914201D3891A0343400886
:1052E00049000028F7D100290AD0914202D10121BA
:1052F000C90705E0914201D2012101E00121C94322
:10530000E005C018401900F0D5FA70BD420005D084
:105310004200120E52428A4201DB00207047C9054A
:1053200008187047F0B507460846584087B0C00FC8
:10533000049048000E46590040084908BC1A8841AC
:1053400005D2384631461E4617460B4602465800DF
:10535000400810434CD0300D039040055900400DDB
:10536000490D0590401A0290402872DA1803012175
:10537000000B09050843019004980092002805D00D
:1053800001995242002088410092019002984021E8
:105390000A1A0199009800F059FA05460C466B4626
:1053A00007CB00F074FAC0197141039A0E0D002367
:1053B000D71756401A467A40164344D0049A002A1A
:1053C0002DD0029A012A039A15DC1205C01A9141C8
:1053D00001263605001C7141D20F059ED2070093AD
:1053E000019202962A46234600F0B2FA07B0F0BDB9
:1053F00038463146FAE71605224A0F46B218C01A57
:10540000B74101210905001C4F4100187F41114699
:1054100018187941E20F10436D19644113E0E20757
:105420006D0815436408C2071443039A0126120548
:10543000C01A91413605001C7141CE074008304327
:105440004908C01851412A46234600F074FACDE7B6
:10545000FFE7049801224000C117121A00238B4174
:1054600004983146C417381AA141EEE730B401243C
:10547000E407634030BC55E730B40124E4076140E1
:1054800030BC4FE70000E0FFF0B51FB488B00B99C7
:105490000998002448400999C00F4900490809911A
:1054A000C0070B990090490049080B910999089889
:1054B000A64608431CD00B990A98084318D00998AF
:1054C00001244000420D4800410D099824050003C5
:1054D000000B204309900B980003000B20430B9016
:1054E00050181C494018002201901446104605E04F
:1054F000002001460DB0F0BD032801DA034600E0AC
:1055000003239C46C11A0AAE0AE05F0008ADED5BBA
:105510004F00F75B7D430027AA187C41491C5B1EA6
:105520006145F2DD410004AB5A522104120C0A43DA
:10553000240C401C0828DFDB01980290009970467B
:1055400001910090059B049A0799069800F000FAD3
:10555000D0E700000DFCFFFFF0B50C465C4085B0C5
:10556000E40FE40703944C000026640859009446B5
:10557000490802460296224321D062460A431ED0C1
:105580006200570D4A000E032303550D0124024605
:105590002C492405781B1B0B360B4018234326434C
:1055A000614600901C46501AB44103D30098401C39
:1055B000009002E0921800985B41002803DA002076
:1055C000014605B0F0BD00200121090507468646C9
:1055D00011E064461D46141BB54106D36546521BB7
:1055E000B341744607430C43A646CD07400849081B
:1055F000284392185B4105460D43EAD110461843F3
:1056000013D06046194650407140084306D06046AA
:10561000101AB34106D20122002306E00022012322
:10562000DB0702E00122D2435310009874460105C3
:10563000381C6141029C039D0019694100F07BF90F
:10564000BFE70000FD03000070B54B005B0803439B
:105650000BD04B005C0D002633466542B341D41796
:10566000AD1AA34102DB0020014670BD12053018BF
:10567000514170BDC217C10F504010B54018CA0744
:105680009623002100F01EF910BD10B500229623CC
:10569000114600F017F910BD0EB5C217C10F5040EA
:1056A000CA0740180021054B0293019200910A4657
:1056B0000B4600F04DF903B000BD000033040000BC
:1056C0000EB505490291002100910A460B46019151
:1056D00000F03EF903B000BD330400004100400279
:1056E0000122400AD205090E80187F2901DA002024
:1056F0007047962903DC9622511AC84070479639A4
:105700008840704770B5CD0F4A0009030123090B8B
:105710001B0519430B4BED070024520D9A4201DA89
:10572000002070BD074B34339A4203DC9A1A00F014
:105730009DF802E00449511888402C43F1D04042C2
:1057400070BD0000FF030000CDFBFFFF4A0009030E
:105750000123090B1B051943094B10B5520D9A4241
:1057600001DA002010BD064B34339A4203DC9A1A4A
:1057700000F07CF810BD03495118884010BD0000AE
:10578000FF030000CDFBFFFFC20FD207400040081F
:105790000BD0C10D0723DB01C91840020905400ADF
:1057A0001143C2084007114370470020014670476B
:1057B00010B5002904DB0124E40740428C41214656
:1057C000002B04DB1C460123DB075242A3418B4222
:1057D00000D1824210BD000010B5002904DB012475
:1057E000E40740428C412146002B04DB1C46012388
:1057F000DB075242A341994200D1904210BD000004
:10580000CB0FDB07490010B5490802460A4307D011
:105810000A0D07240903E401090B121B002A01DC0D
:10582000002010BDC900440F0C43C100E018D20590
:10583000801800F03FF810BD0122D207002800DBDD
:10584000101A002900DB511A8142704710B5202A36
:1058500004DB0146203A9140002010BD91402023F6
:105860009C1A0346E3401943904010BD10B5202A0E
:1058700004DB0846203AD040002110BD0B46D3403F
:10588000D0402024A21A91400843194610BD10B5FB
:10589000202A06DBCB170846203A1041C1170B43DC
:1058A00006E00B461341D0402024A21A9140084341
:1058B000194610BD002904DA401C490001D14008F6
:1058C0004000704770B40024050C05D1102400047A
:1058D00002D1002921D01124050E01D10002083483
:1058E000050F01D10001241D850F01D18000A41CEA
:1058F000002801DB4000641C002908D020252E1B55
:105900000D46F540A14000D001212943084301067E
:105910001B1B000ADB1D02D5002070BC7047DB0595
:10592000181880180029F8DA401C4900F5D170BC1D
:1059300040084000704710B5002B08DA0024401CD6
:10594000614192185B411A4301D14008400010BDEB
:10595000F0B51FB482B005460C0003D0084604F031
:105960008FFC02E004F08CFC2030024600902146BF
:105970002846FFF76BFF049B059A04460F46184321
:105980001143084314D0184610431BD000984021FF
:105990000A1A18460599FFF769FF05460E46009A50
:1059A00005990498FFF752FF084305D0012004E051
:1059B0002046394607B0F0BD0020C11705430E430D
:1059C0002C43374300990E986305401A7905E40A81
:1059D00000220C43FD0A0A3002D500200146E9E707
:1059E0000105101969410C9C0D9D00196941FFF7D3
:1059F000A2FFDFE7FEB500231A461B1A8A4103DB2C
:105A00000020014603B0F0BD4A000D0301212D0B1B
:105A10000905520D0D43D10702D100186D41521EE8
:105A20005110FF31FF310131002704463E46384610
:105A3000009701910246012100200905FFF716FF9A
:105A4000C3197141F818324684468E464A41614670
:105A50002846611A904104D36046241A954176463F
:105A60001F46241900986D41401C00903428E1DD48
:105A7000F91930467041091BA84103D20022D243D4
:105A8000134601E00022134601980105381C7141BC
:105A9000FFF751FFB6E70000064C0125064E05E072
:105AA000E36807CC2B430C3C98471034B442F7D33F
:105AB000FFF70AFB80C30008A0C3000870B58C186C
:105AC0000578401C6B075B0F01D10378401C2A113D
:105AD00006D10278401C03E006780E70401C491C79
:105AE0005B1EF9D12B0705D40023521E0DD40B7079
:105AF000491CFAE70378401CCB1A921C03E01D787E
:105B00000D70491C5B1C521EF9D5A142D8D3002050
:105B100070BD000038B50446064805490068FFF727
:105B2000E7FA604300E0401E00900028FBD138BD3A
:105B300040420F0088010020F8B5044600688168E3
:105B40008907890F012902D10168C90722D181681B
:105B5000114A10261140012500290ED181682943E0
:105B600081600120FFF7D6FF01F062F807460CE0E4
:105B700001F05EF8C01B0A2807D9606D30436065EC
:105B8000A06D2843A0650120F8BD20680068C043CF
:105B9000C007EDD10020F8BD170000801FB50B48ED
:105BA00000900B4801900B4802900B480390694607
:105BB0000A4804F05BFF0A4A08481146083904F015
:105BC00043FE00F0A9FA002004B010BD89C100080E
:105BD00065C10008C5C10008C3C1000894010020C8
:105BE00010000020F8B51848808F00282AD0174CE4
:105BF0000125E16AED051648A94201DB022100E01A
:105C00000021017000F0CAF90126F6020527A082E2
:105C10003F070FE00F4801F025FA80B2A083E18B27
:105C2000421A032A01DC814204D9E0833146384616
:105C300000F0B0F9E06AA842ECDA012231463846B9
:105C400000F0EFFFF8BD0000EC0D00203C0100204B
:105C5000840000200816002010B500231A4603E037
:105C6000845CE3189BB2521C8A42F9D3D84380B2B9
:105C700010BD000010B5034800F096FD024800F08A
:105C800093FD10BD9C1700205417002030B5446CC4
:105C90001C252C400125A540046C656004686360E8
:105CA0008368102B036803D099600068C26030BD20
:105CB0009A600068C16030BD1449012048720A46EC
:105CC00002205E32507203203C3A507204200E3A99
:105CD00050720F480D4B0078087022310870203147
:105CE00008770C495A1C0878587149789971233300
:105CF00018715971203318775977107551751A46F4
:105D00001E3210755175107651767047EC110020D7
:105D10003E0100206401002010B503F0CFFC2020DC
:105D200003F08AFD012005F00BF9002003F084FD4B
:105D3000044804F0A9FF044805F058FA002005F0D3
:105D40008DFA10BD0001002083800000F8B503F03B
:105D500081FD05200121000700F056FF0025144CAD
:105D6000002800D06560134E0221304600F04CFF41
:105D7000002815D1012020700F48808F00280ED0F8
:105D80000127BF0200223946304600F04AFF0A20B0
:105D900004F0CAFC01223946304600F042FF65603B
:105DA000012000F069FE022000F066FEF8BD000050
:105DB0007401002000040050EC0D0020704700002A
:105DC00010B5084900224A6107494B684C15234326
:105DD0004B604B68082423434B60C009C00102603C
:105DE00010BD0000E4170020002002407FB5002510
:105DF0000C460646039500F00FFEE009029003A949
:105E000001960095684600F09FFD002804D000F040
:105E1000D7FD002004B070BD00F0D2FD0120F9E7ED
:105E200010B5002302E0C45CCC545B1C9342FAD34F
:105E300010BD000010B5214A00219069C30520481B
:105E400004D54169022319434161911593699B056A
:105E500005D54369012423434361630219439369D0
:105E60005B0505D54369082423434361E3011943D6
:105E700093691B0505D543690424234343616302E9
:105E8000194393699B0405D5436910242343436157
:105E90006302194393699B0304D5446920231C437F
:105EA000446119439369DB0305D5436940242343C7
:105EB0004361A0020143916110BD00000020024037
:105EC000E417002070B5054600F0B2FE0646184CF7
:105ED0000AE0681C08D0002D04D000F0A9FE801B49
:105EE000A84201D9032070BDA069C007F1D1A06903
:105EF000800701D50220A061A069C00511D4A06966
:105F000080050ED4A06940050BD4A069000508D413
:105F1000A069800405D4A069800302D4A069C003ED
:105F200003D5FFF787FF012070BD002070BD000082
:105F300000200240F8B51746002605460C4600F042
:105F40006BFD09E029460220226800F047FD002889
:105F500004D1241D2D1D361DBE42F3D300F030FDAB
:105F6000BE4201D20020F8BD0120F8BD10B508499D
:105F700002460020054B497905E044001C5B944231
:105F800003D0401CC0B28842F7D310BD901300204C
:105F90007000002010B500F03CFE10BD10B509489F
:105FA00001F060F880B2FFF78BFB074A074BFFF761
:105FB0006BFA0022064BFFF7CFFAFFF7C7FB80B260
:105FC00010BD000008160020F853E3A59B843E4056
:105FD00000408F4070B50024204602F0F1FF474991
:105FE0004748A200641CE4B28150142CF9D34649FE
:105FF00044480A7902754979417544490A7802761C
:10600000497841763F490520133148720A2005F04E
:10601000DDF87D20400105F0F3F83A490022133104
:106020000C2005F0BDF900210C2005F0CBF9384813
:1060300001F018F8344C0125223C2085AD0309E01D
:10604000334801F00FF880B22085E18EFF392D39F9
:10605000884206DBE18E80B28842F1D3491988423A
:10606000EED8022005F002F9002002F0A9FF294D28
:1060700000210F2005F02AF828422064F8D0206C77
:10608000411C38D0400435D58122D20100210F2097
:1060900005F05BF90021102005F018F841061948B9
:1060A000490E0022C73005F047F8164DC735687A0B
:1060B00005281FD102221549681DFFF783F8002823
:1060C00018D11148AE7C66710422691C3630FFF786
:1060D00055F829461331084672000D466930FFF71E
:1060E0004DF860792946420005484838FFF746F8E0
:1060F0000320207070BD04F037F90000FFFF01009D
:10610000F01300204D1200209200002064010020B6
:106110000816002000D0272410B5144C144822463D
:1061200010321146083904F08FFB0022114BE16850
:10613000A068FFF711FA104A104B05F0B5FA0022DB
:106140000F4BFFF799F900220E4BFFF79DF9FFF770
:1061500057FB206000221346E168A068FFF728FB88
:1061600001D0206810BD0020206010BD000000207C
:106170009401002000AA8F406C45D9CC955BC83FA4
:106180000000F03F40A5E54010B5084800F096FA41
:106190000A21064800F032FA044800F01DF9800593
:1061A00003D5024800F01AF980B210BDAC150020EA
:1061B000F8B52F4D00220121284600F032FDFFF7EF
:1061C000E3FFFFF762FA2B4E3146FFF761F82A4CE6
:1061D0000122A0601146284600F023FD2749A0684F
:1061E000002588423EDB2078254F002815D02570F9
:1061F000FFF7CAFFFFF749FA3146FFF749F8A060F9
:10620000FFF7C2FA00223B46FFF730F900221D4B90
:10621000FFF73AF9FFF7F4FA6060A068FFF7B4FA05
:1062200000223B46FFF722F9174A184BFFF72CF9DB
:1062300006460F466068FFF7A7FA134A144B52420E
:10624000FFF722F932463B46FFF76CF8FFF7D8FA22
:1062500010496060884201DD616004E0FF21C905EA
:10626000C84200D365606068FFF738FAC0B2F8BD75
:106270000004005000401B44480000200000604023
:1062800000000C4000E064403333333333B330401C
:10629000CCCCEC3F0000C842F8B50546044640357A
:1062A000287C0026012808D00120287420688168F5
:1062B0008907890F01290ED101E00220F8BD01688C
:1062C000C90708D0606D20210843606501260020C1
:1062D00028743046F8BD616DFF22013291430222DD
:1062E00011436165C1688907890F0091C1688908F8
:1062F0008900C1602068816892071143816000F0C5
:1063000097FC07460EE000F093FCC01B0A2809D951
:10631000606D0221884310210843606500202874C5
:106320000120F8BD206880680028ECDB2068C16887
:10633000009A1143C160606D80088000401C606558
:10634000C5E70000F8B506460D464036317C012908
:106350000DD00121317401688A68520709D5416D59
:10636000202211434165002030740120F8BD022035
:10637000F8BD174B6A68D80547109A42154C8A6ACF
:106380002B6812D05B035B0B1A438A6229684903AE
:1063900005D5A1680143A1600A20FFF7BBFB28686F
:1063A000800312D5A06838430EE05B035B0B9A4371
:1063B0008A622968490302D5A1688143A1602868DF
:1063C000800302D5A068B843A06000203074F8BDF7
:1063D0000110000000270140406D70470068006C0C
:1063E0007047000070B5040006D0606D2646002599
:1063F0004036002802D006E0012070BDA565357446
:10640000204600F0D3F8606DC00603D42168886888
:10641000400705D5606D1021084360653574EBE7D2
:10642000606DFF220132904302221043606588684C
:106430008207920F5B48012A02D10A68D2072BD14A
:10644000032362689B079A4205D05B429A4202D0BE
:106450005B009A4209D10A69920092080A61216898
:106460000A6963681A430A610CE00A69920092089B
:106470000A6181680F229204914381608168626899
:10648000114381602168CA6818239A43CA60216851
:10649000CA68A3681A43CA60816801225206914300
:1064A00081608168A28E52061143816020688168F4
:1064B000C90004D481680122120711438160206859
:1064C000C168394A1140C1602069E168022825D0BD
:1064D00000200143204620300278037B52035B00FA
:1064E0001A431143226B1143A26992031143E269DB
:1064F000D20311432268D3681943D160616A0A4606
:10650000FF3AC23A05D0A26A11432268D368194300
:10651000D16042780121012A02D00BE00420D8E7A3
:106520000078002823D0606D202210436065A06DA4
:106530000843A065E06B012820681FD00169C907E6
:1065400003D0016949084900016120684169C9080F
:10655000C900416120684169A26B11434161A56591
:10656000606D80088000401C6065002070BD206860
:10657000C26801231B041A43C260DBE70269FF23E0
:106580009B009A43026120680269236CA66C1A433F
:10659000636C33431A430261206802690A43026153
:1065A000D3E70000002701401902FEFF10B586B0B6
:1065B000044614216846FEF7FAFD0E492068884219
:1065C00016D10D48416B421511434163C16A012246
:1065D0001143C162C06A69461040059002200090D4
:1065E00003200190002002900520000700F050FADF
:1065F00006B010BD0024014000100240F8B504466A
:106600004069254640350E4608280BD02068C068F2
:10661000C00709D0606D2021084360650020287400
:106620000120F8BD082700E00C2700F001FB0090D6
:1066300011E0701C0FD0002E05D000F0F9FA00997F
:10664000401AB04207D9606D0421084360650020FC
:1066500028740320F8BD206800683842E9D0606DD6
:1066600001214902084360652068C16809058A0F55
:106670000C21002A1BD12022125D002A17D10268AA
:10668000120714D5826853070122002B08DB4368E8
:106690008B434360606D130298431043606506E0CE
:1066A000606D202318436065A06D1043A065A0694C
:1066B000002801D1206801600020F8BD70B50446B3
:1066C000216800208968490721D425464035297C66
:1066D00001291CD001212974E169012904D0204637
:1066E000FFF72AFA002811D1616D0A4A1140FF22F2
:1066F0000132114361650021A165297422681C21C2
:10670000116021688A6804231A438A6070BD0220E0
:1067100070BD0000FEF1FFFF30B5014620314A791F
:106720000023022A04D00422C2630B71012030BD71
:10673000026814680E25AC4314600268146864088B
:1067400064001460446C1C22144001221546006C45
:10675000A54045604A7118460B7130BD70B50024E4
:10676000014620314A79022A03D00421C163012461
:1067700018E0026813680E25AB43136002681368C3
:106780005B085B001360436C1C221340012215461A
:106790009D40036C5D604A7100220A71816B002983
:1067A00000D08847204670BDF0B4016C0D680168C8
:1067B0000C68466C1C2304221E401746B7402F422B
:1067C0000ED067070CD50C68A40602D40C6894435D
:1067D0000C60416C19408A40016C4A60016B1AE000
:1067E0000227B74002462F402032002F17D0A707BC
:1067F00015D50C68A40605D40C680A25AC430C60BA
:1068000001215171446C02211C40036CA14059606C
:1068100000211171C16A002918D0F0BC084708276F
:10682000B7402F4212D0240710D50C680E25AC4378
:106830000C60446C01211C400B46A340046C636057
:10684000C163517100211171416BE4E7F0BC7047E5
:1068500070B504003CD01F48256814212818FEF7A5
:1068600047FC800060641C482064022120462030E0
:106870000246417129681948E3680140A0686669C9
:106880001843236933431843A3691843E369184342
:10689000236A1843084328600121A06889038842BD
:1068A00010D00D488030836A656C1C210D400F2686
:1068B000AE40B3438362656C63680D40816AAB4050
:1068C0000B4383620020E06301215171107170BDA0
:1068D000012070BDF8FFFDBF000002400F80FFFFE8
:1068E000F8B504468C46203001790025012909D0ED
:1068F0000126067141790027012905D0077102257B
:106900002846F8BD0220F8BD02214171E7632068E6
:10691000016849084900016061462046FFF7B6F961
:10692000206B00282068016801D00E2205E00422B7
:1069300091430160206801680A22114301602068C8
:10694000016831430160DBE7F8B51A4E0546307C3B
:106950000F46012807D0012030741748FFF7B2FA1C
:10696000010002D021E00220F8BD0020C0433860C1
:106970006C6814E02046FFF723FA0F48FFF7A2FAED
:1069800001460E48426808239A4342604268431514
:106990009A434260002901D03C6006E08034A86838
:1069A0006A68C0018018A042E4D80020307408460C
:1069B000F8BD0000E417002050C300000020024092
:1069C0000548416802221143416041680122114398
:1069D000416000207047000000200240F8B50C4CD8
:1069E0001646207C0F46012808D001202074094853
:1069F000FFF768FA0025002802D006E00220F8BD63
:106A000065613E600348FFF75DFA2574F8BD00003C
:106A1000E417002050C3000011484168C9070BD09B
:106A2000EFF3108172B60F4AC2600F4AC26081F361
:106A300010884168C9070ED1416889070DD5EFF369
:106A4000108172B6094A0261094A026181F3108815
:106A50004068800701D50120704700207047000082
:106A600000200240EFCDAB8905040302BFAE9D8C30
:106A7000161514137047000010B504494A69024204
:106A800002D04861FFF7F6FF10BD0000000401408E
:106A9000FCB500230124A2E027462A469F403A4045
:106AA0006FD04D68012D05D0022D03D0112D01D0DE
:106AB000122D16D185680326AC465D00AE46AE4069
:106AC0006546B543AC46CE687546AE4065462E4336
:106AD000866046680D79BE43ED06ED0F9D40354357
:106AE0004560C6685F000325BD40AE46AE433546EF
:106AF0008E68BE402E43C6604E68022E01D0122E14
:106B000014D1DE08B60036180196366A5D07B44621
:106B1000EE0E0F25B54000966646AE43B4460D69AD
:106B2000009EB54066462E43019D2E62066875465E
:106B3000AE430D79AD07AD0FBD40354305604D68DF
:106B4000ED004BD5294D6E6B26436E639E08284D94
:106B5000B6007519AC46AD689E07360F0F27B740D3
:106B6000BD4305273F07B84201D1002715E0214F5B
:106B7000B84201D1012710E01F4FB84202D10227CD
:106B80000BE02BE01D4FB84201D1032705E01C4F5D
:106B9000B84201D1052700E00627B7402F436546DC
:106BA000AF60184D2E684F689643FF0300D516431B
:106BB0002E606E684F689643BF0300D516436E6023
:106BC000AE684F689643FF0200D51643AE60EE688C
:106BD0004F689643BF0200D51643EE605B1C0A68FF
:106BE0001546DA4000D057E7FCBD00000010024017
:106BF000000001400004005000080050000C00504C
:106C0000001C0050000401400069084000D0012031
:106C10007047426913460B401B0491430B43836149
:106C20007047002A01D0816170478162704700007F
:106C300001488068704700007C010020024881689C
:106C400002788918816070477C01002010B50848DF
:106C500000240168402211430160204600F00AF838
:106C6000002801D0012401E000F046FA204610BDC2
:106C70000020024070B504460D4D7D202978C000EB
:106C8000FEF736FA01460B480068FEF731FA00F0CD
:106C90002FFF002809D1042C07D200222146401ED4
:106CA00000F052FA00206C6070BD012070BD000041
:106CB0007C0100208801002070477047F8B502F081
:106CC000C9FD624C0120E070208AFEF7DEFC01461F
:106CD0007F20C005FEF7DCFA5D4D06462968FEF709
:106CE0007EFA28600120E56AC005854201DA28465F
:106CF00007E030460121FEF709FB2946FEF7C4FAFA
:106D0000E062FF21C9050025C84200D3E562607832
:106D100000280BD102214F48FFF776FF02004E49B1
:106D20004E4817D00022FFF77CFF25630221494817
:106D3000FFF76AFF4A4E002855D02563B08AFEF758
:106D4000A4FC434F3968FEF777FD5FD24549012027
:106D500008705DE00122D1034048FFF762FF208AFE
:106D6000FEF793FC01467F20C005FEF791FA216BE8
:106D7000FEF735FA3C4920638842D7DD38480127C1
:106D8000F926403000900A213046FEF7B1F900297B
:106D900003D131493148FFF7FDF802212D48FFF7B3
:106DA00033FF002801D0002701E0002F12D102217B
:106DB0002848FFF729FF00280CD104F03DFC00997A
:106DC0000120888005F094F9642003F0ADFC284987
:106DD0002648C8600A2003F0A7FC3046761EF6B2AB
:106DE0000028D0D1A2E7208AFEF74FFC01467F2081
:106DF000C005FEF74DFA216BFEF7F1F91D4920633E
:106E000088429BDB1A491948C86097E71548057006
:106E1000708F401EFEF72EFC3968FEF70DFD06D878
:106E20002079002803D014490120087001E012489D
:106E30000570708FFEF729FC3968FEF7FDFC04D25F
:106E40002079002801D004F0B9FBF8BD3C010020F6
:106E50007801002000040050008000000000005075
:106E6000EC0D002076000020000040400400FA05F0
:106E700000ED00E00000A04086000020704770B5E3
:106E8000040010D0022025462035A873204601F0CA
:106E900057FBA87B032805D0204600F0B9F8002056
:106EA000A873687370BD012070BD7047704710B53E
:106EB000044600680168C943C90708D18168C9430D
:106EC000C90704D1012141602046FFF7F7FE206881
:106ED0000168C943890708D48168C943890704D474
:106EE000022141602046FFF7E7FE20680168C943A0
:106EF000490708D48168C943490704D40421416083
:106F0000204600F0F7F820680168C943090708D453
:106F10008168C943090704D4082141602046FFF76E
:106F2000ADFF20680168C943C90608D48168C94318
:106F3000C90604D4102141602046FFF7BEFE206838
:106F40000168C943890608D48168C943890604D405
:106F5000202141602046FFF7A9FF20680168C9434E
:106F6000490608D48168C943490604D440214160D8
:106F70002046FFF79AFF10BDF8B5040005D025465E
:106F80002035A87B002802D006E00120F8BD0020B3
:106F90006873204600F04EF80220A8732068C2688B
:106FA00084466368012B01D106208243164861693B
:106FB000814202D0072040038243002B01D1D82018
:106FC00082431248A668024018463043676A266A20
:106FD0003E433043A66A30431043002B02D0012BBE
:106FE00004D005E02369E2691A4300E0E268104337
:106FF000054A914202D0A269114308436146C86024
:107000000120A8730020F8BDFFFF0000F8F119FF70
:1070100010B500680549884207D10548816B4900D1
:10702000490881630D2000F073F810BD007C00401A
:107030000010024010B50068084988420CD1084889
:10704000816BC20411438163002201210D2000F0F5
:107050007BF80D2000F06CF810BD0000007C0040B3
:10706000001002400068C06970470000F8B504468F
:107070000220254620351746A8731D480268C30420
:107080001A4302602068C2689B121A43C2602068DB
:107090000269012632430261226810205060206894
:1070A00081611021204601F0BBFA03281FD021681E
:1070B00008204860206847610821204601F0B0FAA6
:1070C000032814D0204601F03BFAA87B03280ED0F9
:1070D0002068816831438160206801693143016122
:1070E00020680169042211430161AE730020F8BDDC
:1070F00000040140704700000448416B0122114325
:107100004163816B020411438163704700100240A8
:10711000002809DBC106C90E012088400349086028
:10712000BFF34F8FBFF36F8F7047000080E100E027
:10713000002805DBC106C90E01208840014908600E
:107140007047000000E100E010B503F0EBF810BD5F
:1071500002494A6882434A6070470000007000405C
:1071600002480168821511430160704700700040B9
:1071700002494A6802434A607047000000700040BC
:107180000548016802221143016004480169042294
:107190001143016130BF70470070004000ED00E016
:1071A000F0B5154A1368154D54152D6A2340ED07A7
:1071B000ED0F002B04D0002D02D01668A6431660F8
:1071C0001668B608B600064316600D48076904261F
:1071D0003743076101290DD040BF20BF20BF01699F
:1071E000B1430161002B04D0002D02D01068204370
:1071F0001060F0BD30BFF2E70070004000000140B9
:1072000000ED00E0F8B5044600780027534D8006F5
:1072100071D5524E403EB06BC00004D4B06BA9058E
:107220000843B06301274E480168C90511D40168BD
:10723000821511430160FFF7FBFC009005E0FFF7AA
:10724000F7FC0099401A642837D845480068C00503
:10725000F5D532680321090560680A400140914272
:1072600008D08103890F032904D13168890301D52E
:107270000120F8BD2A69032109040A4022D00840F0
:1072800090421FD0207880061CD528692A6988433F
:107290000121C9040A432A612A698A432A612861B3
:1072A000C0050FD5FFF7C4FC009008E0FFF7C0FC55
:1072B0000099411A2B48814201D90320F8BD286961
:1072C0008005F3D561688803800F032805D13268F3
:1072D0000005824301400A43326028690322616845
:1072E0001204114008432861002F04D0B16B012023
:1072F00000078143B1632078C00705D0E868A16822
:10730000800880000843E8602078800705D5E86899
:107310000C218843E1680843E8602078400706D5DF
:10732000E86803218902884321690843E8602078DE
:10733000000706D5E868032109038843616908430B
:10734000E8602078000606D5E868032189048843B0
:10735000A1690843E8600020F8BD00004010024029
:107360000070004088130000F8B50E46050038D0C4
:107370005E480068C007C00FB04214D25B4C206862
:107380004008400030432060FFF752FC074605E00C
:10739000FFF74EFCC11B564881427AD82068C007CF
:1073A000C00FB042F4D12878524C800705D5E06870
:1073B000F0218843A9680843E0602878C00752D0CC
:1073C0006868022806D0032807D0216801280AD05F
:1073D000890504E02168890301E021688901002909
:1073E00003DB0120F8BD4907F9E7E1688908890056
:1073F0000143E160FFF71CFC0746686802280AD0D9
:10740000032814D001281ED029E0FFF711FCC11B6E
:10741000374881423DD8E0680007800F0228F4D148
:1074200021E0FFF705FCC11B3148814231D8E068FB
:107430000007800F0328F4D115E0FFF7F9FBC11B0B
:107440002B48814225D8E0680007800F0128F4D13D
:1074500009E0FFF7EDFBC11B2548814219D8E06820
:107460000007800FF5D121480168C907C90FB14253
:1074700017D901684908490031430160FFF7D8FB7B
:10748000074608E005E0FFF7D3FBC11B184881421F
:1074900001D90320F8BD15480068C007C00FB042ED
:1074A000F1D12878400706D5E06807210902884312
:1074B000E9680843E0602878000707D5E0680721FD
:1074C000C90288432969C9000843E06000F03AF81E
:1074D000E168094A0906090F515CC840074908607C
:1074E00007480068FFF7C6FBF8BD00000020024017
:1074F0008813000000100240CAC200088801002062
:1075000080010020044805490068C968044A49050B
:10751000490F515CC84070478801002000100240AC
:10752000E3C20008044805490068C968044A8904A0
:10753000490F515CC840704788010020001002408C
:10754000E3C2000870B51A4AD3681A490C201840E3
:107550008D0004280CD04E00082810D00C2810D024
:1075600050680004410F0120C003491C884070BDD1
:107570001068C00601D5084670BD284670BD30466B
:1075800070BD98020C4C000F205C1B029C0FD3684E
:10759000641CDB0301D5314603E01268D20600D437
:1075A000294602F084FE22460023FDF7B7FD70BD98
:1075B0000010024000093D00DAC20008FEB50500D7
:1075C0007ED0FE4CE7680C20E668074001200004EE
:1075D00006402878C00747D0082F05D00C2F0AD1C5
:1075E00001200004864206D1206880033CD56868EB
:1075F0000028E5D038E0012069680004814203D109
:1076000021680143216011E0052301221B0492043B
:107610009942216802D111432160F1E78143216041
:10762000216801400091206890432060686800282C
:107630000DD0FFF7FDFA009005E0FFF7F9FA009989
:10764000401A64287BD820688003F6D50CE0FFF749
:10765000EFFA009005E0FFF7EBFA0099401A642872
:10766000F0D820688003F6D42878800756D50923FF
:10767000E868042F0DD00C2F01D1002E09D000286E
:107680003CD02168994301432160FFF7D1FA0646B7
:1076900028E02168490701D5002891D061681F22A0
:1076A000120291432A6912021143616021689943D1
:1076B00001432160FFF746FFE16809060A0F00E079
:1076C0008BE1BF49895CC840BE490860BE4800687C
:1076D000FFF7D0FA002873D120E0FFF7A9FA801B4A
:1076E0000228AFD820684007F7D560681F2109023B
:1076F000884329690902084360600FE02068400858
:1077000040002060FFF794FA064604E0FFF790FA85
:10771000801B022896D820684007F7D42878C00636
:1077200060D5002F0CD0A86900284AD02068FF211E
:10773000013108432060FFF77BFA06462EE0C1E0E6
:107740002068800502D5A8690028A6D060680721B6
:1077500049038843296A084360606068297F000202
:10776000000A090608436060286A410B0120C00333
:10777000491C8840E16809060A0F9149895CC840A4
:107780009049086090480068FFF774FA002817D104
:1077900028E0FFF74DFA801B0228A2D82068800558
:1077A000F7D56068072149038843296A0843606068
:1077B0006068297F0002000A09060843606011E042
:1077C000E2E02168FF20013081432160FFF730FAB9
:1077D000064604E0FFF72CFA801B022872D82068C6
:1077E0008005F7D42878794E000724D568690028E9
:1077F000306910D0012108433061FFF719FA009079
:1078000005E0FFF715FA0099401A02285AD83069A6
:107810008007F6D50FE0400840003061FFF708FA16
:10782000009005E0FFF704FA0099401A022849D8B1
:1078300030698007F6D42878400766D5002002908A
:10784000A06BC00006D4A06B012109070843A06308
:10785000012002905E480168C90511D401688215B3
:1078600011430160FFF7E4F9009005E0FFF7E0F94C
:107870000099401A642825D855480068C005F5D5F8
:10788000FF20AA680130824203D13169014331618E
:1078900011E001218902002A07D005231B029A4228
:1078A00003D132690A433261EFE7326982433261C0
:1078B000306988433061A868002810D0FFF7B8F914
:1078C000009008E05FE0FFF7B3F901460098091A5D
:1078D0004048814257D830698005F4D50DE0FFF764
:1078E000A7F9009006E0FFF7A3F90099411A39487B
:1078F000814248D830698005F5D40298002804D028
:10790000A06B012109078843A063686A002866D03C
:107910000C2F3ED0012636060228206805D0B04341
:107920002060FFF785F905462FE0B0432060FFF7A0
:107930007FF9074604E0FFF77BF9C01B022822D835
:1079400020688001F7D4E96AA86AE2680843296BD5
:10795000FD231B049A4311430843E0602068304331
:107960002060FFF765F9054604E0FFF761F9401B69
:10797000022808D820688001F7D530E0FFF758F9D1
:10798000401B022801D90320FEBD20688001F5D4E8
:1079900025E00128F8D0E06801210904AA6A014025
:1079A00091421AD10F218904EA6A0140914214D10F
:1079B000032189050840296B88420DE00010024030
:1079C000CAC2000888010020800100204010024047
:1079D000007000408813000001D00120FEBD00208F
:1079E000FEBDF8B504000ED0FF27606A05370025FC
:1079F00000280AD02561656126464036A562707C64
:107A0000002807D00AE00120F8BD6068B842F3D032
:107A1000E561F1E73574204600F03EF8022171740B
:107A20002068026840239A4302602123A2686068AC
:107A30009B021A4038401043E3688A0213401843FF
:107A400023690B40217D1843C907C90F0843A16969
:107A5000931019400843E169382319400843216A0B
:107A6000802319400843A16A930019400843216804
:107A70000860A0690421000C0840616A10231940C5
:107A80000843216848602068C1699143C161656508
:107A9000012070740020F8BD10B586B00446142192
:107AA0006846FDF784FB10492068884219D10F48C9
:107AB000416B821411434163C16A01221143C162C7
:107AC000C06A002110400590E02000900220019043
:107AD0000320039002910491052069460007FEF7F8
:107AE000D7FF06B010BD000000300140001002407A
:107AF000094910B5401E884201D9012010BD074C2C
:107B000060610321081F02F00DFC0020A061072026
:107B10002061002010BD0000FFFFFF0000E000E03A
:107B20007047704770470000F8B502680446D06996
:107B300011689668814B05461D402023002D6CD0AE
:107B4000F7077F4DFF0FBC460D402F4379D02546E8
:107B5000C7078035002F06D0CF0504D5012717624F
:107B60002A683A432A60820708D5F20706D02768B8
:107B700002223A622A6804273A432A60420708D55B
:107B8000F20706D02668042232622A6802263243AF
:107B90002A6002070AD50A461A406646324305D0D3
:107BA0002668082232622E6816432E60020508D528
:107BB0004A0106D501222668D20232622A681A4397
:107BC0002A602A68002A30D0800606D5880604D5A7
:107BD000616E002901D0204688472868216889689D
:107BE000490602D42821084225D0204602F0ABF8ED
:107BF00020688168490619D5826840218A438260DD
:107C0000206F002812D04F498163206FFEF7A6FD38
:107C100000280AD0206F816B06E0850611D58D06FD
:107C20000FD5616E77E020468847F8BD2046FFF704
:107C300079FFF8BD05E02046FFF774FF00202860BB
:107C4000F7E7256E012D56D1C50654D5CD0652D580
:107C500010261662206881682546490640350029AD
:107C60002ADA226F116849680904090CE1D02F8BC8
:107C70008F42DED9698311680968890617D40168C3
:107C800032019143016020688168490849008160A0
:107C900020688168402291438160E367002020666C
:107CA00020680168B1430160206FFEF735FD288B25
:107CB000698B401A81B21AE0298B6A8B891A6A8B08
:107CC00089B2002AB5D00029B3D00268FF2521353A
:107CD000AA43026020688268520852008260E3670B
:107CE00000202066606620680268B2430260204679
:107CF000FFF716FF9DE7C50208D5750206D50120DE
:107D0000000510622046FFF70CFF92E7050605D537
:107D10000D0603D5A16E002985D18AE7400688D5D6
:107D2000480686D5116820464024A1431160836728
:107D30000021816600F043F97BE700000F08000096
:107D4000200100046D9C000810B5040003D0A06F52
:107D5000002802D007E0012010BD00217420015549
:107D6000204600F027F82420A06720680168490811
:107D700049000160204602F039F80128ECD0606A21
:107D8000002802D0204601F05BFE206841680922ED
:107D9000D20291434160206881682A229143816028
:107DA00020680168012211430160204601F0AEFE07
:107DB00010BD0000F0B587B0064614216846FDF7F7
:107DC000F6F92C493068884251D12B48416B012289
:107DD000920311434163C16A01221143C162C06A27
:107DE0000025104005900320400200900220032748
:107DF00001A9A1C104200490052069460007FEF7EF
:107E000047FE1F4C1D48A560E56081C48027E560E2
:107E1000A7602020256160610002A0611848083C2D
:107E2000FEF716FD002801D0FDF7C8FF3467A662F3
:107E3000144C124821461438206003206060102042
:107E40000831A1C16561A561E56120462562FEF7A3
:107E5000FFFC002801D0FDF7B1FFF46600220121EC
:107E60001B20A662FFF770F91B20FFF761F907B02E
:107E7000F0BD000000380140001002403000024018
:107E8000541700209C17002070B5C36F202B27D1FA
:107E900000290BD0002A09D0012483682403A342BF
:107EA00006D10369002B03D1CB0701D0012070BD9F
:107EB000034660331C7D012C12D001241C75002365
:107EC0000366084C0368A34207D05C68240204D50B
:107ED0001C680125AD062C431C6002F087F870BDBC
:107EE000022070BD0048004070477047FFB504464F
:107EF000806F83B017460D4620285ED1002D0AD032
:107F0000002F08D0A168C001814207D12069002854
:107F100004D1E80702D0012007B0F0BD2046603050
:107F20000090007D012848D00098012101750020B3
:107F3000802108512120A067FEF77AFE26464036B0
:107F40000190378277820120A1680003814202D12B
:107F50002069002805D02F460025009900200875CB
:107F600011E00027F9E700228021204602F084F882
:107F7000002815D1002F15D02168387888627F1C21
:107F8000708A401E7082708A019B002806980090BB
:107F9000E9D100224021204602F06EF8002808D0E6
:107FA0000320B9E728882168C005C00D8862AD1C90
:107FB000E6E72020A0670020AEE70220ACE770478C
:107FC000034D044C04A002F051F9E560FAE700000B
:107FD0000400FA0500ED00E0486172644661756CCA
:107FE000745F48616E646C65722E0D0A00000000BB
:107FF00070B586B014216846FDF7D9F801240B4806
:108000000526C4800A48E5024483360722462946ED
:108010003046FEF706FE002102910391009501947F
:1080200069463046FEF734FD06B070BD2C0E0020C8
:108030003C01002070B501240E4DA403002221460E
:108040002846FEF7EEFD002204212846FEF7E9FD52
:108050000A2002F070FB012221462846FEF7E1FDCE
:108060000A2002F068FB002221462846FEF7D9FDCF
:1080700070BD00000004005070B501240E4DA40333
:10808000002221462846FEF7CCFD01220421284685
:10809000FEF7C7FD0A2002F04EFB012221462846CA
:1080A000FEF7BFFD0A2002F046FB002221462846CB
:1080B000FEF7B7FD70BD000000040050F1B50024CC
:1080C0000126154F2546B603002231463846FEF7F5
:1080D000A8FD0A2002F02FFB012231463846FEF7A8
:1080E000A0FD6006040E04213846FEF78DFD002831
:1080F00001D0641CE4B2052002F01DFB6D1CEDB242
:10810000082DE1D30098002803D0FFF793FF204605
:10811000F8BDFFF7B1FFFAE700040050F8B50126FB
:10812000154F0546B603002231463846FEF779FD65
:108130000024E80901D0012200E000220421384691
:10814000FEF76FFD6806050E0A2002F0F4FA012220
:1081500031463846FEF765FD0A2002F0ECFA0022AF
:1081600031463846FEF75DFD0A2002F0E4FA641C51
:10817000E4B2082CDDD3F8BD0004005070B50D4CFE
:10818000012204212046FEF74CFD012295032946D9
:108190002046FEF746FD002204212046FEF741FD61
:1081A0000A2002F0C8FA002229462046FEF739FDCF
:1081B00070BD00000004005070B501240E4DA403F2
:1081C000002221462846FEF72CFD002204212846E5
:1081D000FEF727FD0A2002F0AEFA012221462846CA
:1081E000FEF71FFD012204212846FEF71AFD0A2092
:1081F00002F0A1FA70BD00000004005070B5144DEB
:108200000024012204212846FEF70BFD062002F07F
:1082100092FA0122960331462846FEF702FD062017
:1082200002F089FA07E0641CE4B2FA2C03D9FFF7E4
:10823000C3FF012070BD04212846FEF7E5FC00289D
:10824000F1D1002231462846FEF7EBFC002070BD3C
:1082500000040050F8B501F08BFC01F0BBFC3B487A
:108260000068C069FDF7A4FF394D3A4E28704021DF
:108270003046FEF7C9FC77010024002827D0364895
:108280000460A879002803D10120A87101F056FFED
:1082900080213046FEF7B8FC002806D000220821D5
:1082A0003046FEF7BEFC012205E0012208213046DF
:1082B000FEF7B7FC0022052039460007FEF7B1FCA7
:1082C000264D274EA88C274F012803D01CE0AC7107
:1082D0000022EBE724486946088072B680212348D3
:1082E000FDF784FD002804D0022269461F48FDF7EF
:1082F00021FE62B61EA001F0B9FFAC8403F0F8FEC7
:10830000642002F011FAFE60688C012809D113483C
:108310006C844038048003F0EBFE642002F004FA21
:10832000FE60288C012806D12C8403F0E1FE642035
:1083300002F0FAF9FE600948114A4038018891427A
:1083400002D1C088002800D1FE60F8BDD016002000
:108350003C01002000040050780100202C0E002079
:108360000400FA0500ED00E0AAAA0000384A00085F
:10837000BDF8C8EBC9FDBCB6C4A3CABD0D0A000058
:10838000AA55000038B500246946202000F0AAF85C
:1083900068460078572800D001246946212000F063
:1083A000A1F868460078032800D0012469462220FD
:1083B00000F098F868460078402800D0012469460B
:1083C000232000F08FF868460078082800D00124A8
:1083D0006946302000F086F868460078AA2800D068
:1083E00001246946322000F07DF80C486946008F70
:1083F0000978884200D001246946332000F072F8E1
:1084000006486946403040880978884201D1002CEE
:1084100002D004490248C86038BD0000EC0D0020BD
:108420000400FA0500ED00E038B55721202000F0E7
:108430007AF80321212000F076F84021222000F074
:1084400072F80821232000F06EF8AA21302000F0F5
:108450006AF81048018F142901D8002901D101219F
:1084600001870C4C40346188142901D8002901D1BE
:1084700002216180008FC1B2322000F054F8A1784F
:10848000332000F050F8684600F006F80A2002F0A9
:1084900052F938BDEC0D002010B501460F2000F058
:1084A00021F8002800D0012010BD10B50446FFF7C8
:1084B00065FE3220FFF732FEFFF7A0FEE0B2FFF7C5
:1084C0002DFEFFF79BFEFFF759FE3320FFF726FE38
:1084D000FFF794FE0020FFF7F1FD0446FFF76CFE66
:1084E000204610BD10B50C46FFF7DFFF20700120BD
:1084F00010BD70B50D460446FFF740FE3220FFF771
:108500000DFEFFF77BFEE0B2FFF708FEFFF776FEF9
:108510002846FFF703FEFFF771FEFFF74DFE0A2026
:1085200002F009F970BD10B5FFF7E3FF012010BD9F
:1085300010B50248FEF7BBFC10BD00000816002075
:10854000FEB50446002772B6334A01688B1804D181
:108550003248C76803208004074088680190C868D3
:10856000009048698E69002B08D12C4940398B6AEC
:10857000CD042B438B628B6AAB438B620146314344
:108580003CD025492368CB4205D12449CA6803233E
:108590009B049A43CA6025462035002810D02168E4
:1085A0000A6901231A430A612168486108212046AB
:1085B00000F036F8032800D1A8732168082048602D
:1085C000002E10D02068016901221143016120684A
:1085D00086611021204600F023F8032800D1A873FB
:1085E0002168102048600C482168C14206D10B4820
:1085F000C1680322920491433943C1602068016934
:108600004908490001612168019888602168009843
:10861000C86062B6FEBD00000084FFBF401002408B
:1086200070B506460B480D46002409490068FCF762
:108630005FFD7D21C90048433168401E00D10324FD
:108640000B682A469A4301D00028F6D1204670BD17
:10865000204E0000880100201CB500211648009122
:10866000144A01910260C1631205426081600722D1
:108670008263012202610246C16020321170FF2331
:108680005170C233436281621173016381610422BC
:1086900041634261C161FDF7A5FE08480090801367
:1086A000019069460448FDF74DFE00210248FDF7A0
:1086B000F3FD1CBD00240140AC15002002000004A5
:1086C00008B50848016B012211430163006B0121C9
:1086D0001040009000220A20FEF736FD0A20FEF727
:1086E00027FD08BD00100240F0B587B01421684690
:1086F000FCF75DFD4648C26A04210A43C262C26AB1
:108700000A400592C16A80263143C162C16A314084
:108710000591C16A01242143C162C16A21400591CA
:10872000C16A02252943C162C06A224628400590D9
:10873000052010210007FEF774FA0122354936485A
:10874000FEF76FFA002235493348FEF76AFA9121A5
:108750000520002209020007FEF763FA3048019065
:10876000002705206946029700940007FEF790F95C
:108770002C48009011200190032003900297694635
:108780002548FEF785F910206A46039591C2052019
:1087900069460007FEF77CF91120019002976946AF
:1087A000039700941C48FEF773F91F48019069462F
:1087B000009502941848FEF76BF940200090694636
:1087C000019702951448FEF763F91848694691C16C
:1087D000694611480397FEF75BF99120000269464C
:1087E00091C10520694600070397FEF751F96946D4
:1087F0000948019700960294FEF74AF900220121E8
:108800000520FEF7A1FC0520FEF792FC07B0F0BDA5
:108810000010024005420000000400500830000033
:108820000000111004400000000021100832000078
:1088300010B50F4C0D482060FF200530606000200F
:10884000A060E06020616061E06101212062490276
:108850006062A161A0620720E0622046FFF7C1F8D4
:108860002068016840221143016010BD00300140C2
:108870003816002000B585B014216846FCF797FC37
:108880000E480D490160E1214902416000218160EB
:10889000C160016181610C22C161426101623021CC
:1088A00041620121090381634900C163FFF74CFA6A
:1088B00001F03EFC05B000BD00380140D01600209C
:1088C00070470000F0B589B00A2002F07FFC7D20DF
:1088D000400102F095FCFF4C0025A570FE48206683
:1088E000607C0C2801D30B20607460790A2801D9C0
:1088F0000A206071F948E570F94E00783071F94945
:10890000A079097840000843A17D89000843F071EF
:10891000E06BF070010A3172401CE0636079B07462
:1089200042003046F0491330FCF728FC6079EE49EC
:1089300082004000801960311330121DFCF71EFCCC
:1089400060790621420048438019E8491730921C9B
:10895000FCF714FC2E20205E002803D0E449098A8D
:108960000818E0856079DB49C000223182190B7B51
:1089700053764B7B937606227272DE4A1D30127854
:10898000B272A28C3273D64A0B79133A13754979B5
:1089900051750022D24902F003FD60790021C00028
:1089A0001D3002F00FFDD448FEF75CFB0127208547
:1089B000BF0309E0D048FEF755FB80B22085E18E69
:1089C000FF392D39884206DB81B2E08E8142F1D336
:1089D000C0198142EED8022002F048FCC0480126AE
:1089E000C571A574A5732674E573C348FEF73AFBF9
:1089F00060850746E5706079FCF762FEBF4AC04BB0
:108A0000FCF742FD01F02CFE0022BE4BFCF78AFC75
:108A1000FCF79CFE0006C00CC01980B2F103A085D3
:108A2000884201D3401AA085B748E0642079401CF1
:108A30002071B148FEF716FB2085AB48A54F64387E
:108A400040370690B1E1AC48FEF70CFB20850BE007
:108A5000A948FEF707FB80B22085A18D884203D389
:108A6000AA4A8918884207D300210F2002F02EFB62
:108A7000A74920640842EBD0206C411C1FD0400461
:108A80007ED58122D20100210F2002F05EFC002160
:108A9000102002F01BFB41069348490E00227C384F
:108AA000E16502F049FB002002F0AAFB002002F081
:108AB0005CFB8D487C38417A0729C3D101E001F085
:108AC00053FC02229349401DFCF77CFB0028B9D1DE
:108AD00002F0C9FCE167A06702F0B2FC7D4B803375
:108AE00003C3E0788049401CE07083390B7A684604
:108AF0000370497A417000880390E18C88427DD1EF
:108B0000774985488C31C98E0180754871498C3010
:108B1000008F48847848FEF7A5FA208502F0E8F92E
:108B20006C48FF2280300168406852040023891895
:108B300058410206080A10434108490000900A0EF5
:108B4000080264498031CA6088606548E36F0A3072
:108B5000A26F02F05DFC60798100614808185D49F0
:108B6000163080310CC902F053FC5A488030C3687B
:108B700082685B48123002F04BFC0821584800E044
:108B800006E14172B430C07C0009607514D05648CB
:108B9000022260497738FCF715FB00280CD15048B9
:108BA000A674C671E06D50491638C2B26639C81D48
:108BB000E274FB30FCF7E2FA607900228000484959
:108BC0001C3002F0EDFB6079002180001C3002F0C7
:108BD000F9FB009802F0F3FA012002F047FB207342
:108BE00002214E48FEF710F800281DD000213D4814
:108BF00001703B498C31488E049000E05AE0388186
:108C0000888E78818446A06CFF310531E06408606D
:108C1000DC392065C97C0907090F032900D02175BB
:108C2000E16D1C2902D015E00121E0E72C49294A19
:108C30008C31C98F1186069B2C4A1B881380884271
:108C400007DD002805DD002903D0207E401C2076AA
:108C500000E025762571A6730498B8816046F881F6
:108C6000E673608C2E49FF30C33080B26084884246
:108C70000CD949424018608427487D220188D200DF
:108C8000491C89B20180914200D3058022487D2190
:108C90000088C9004843618C4018606500F076FD8B
:108CA000207B002805D100210F2002F00FFA0006DA
:108CB000F9D583E0FDF75AF90B4A0321903211549C
:108CC00007498C314A8E3A81898E7981E26D1C2A5E
:108CD0002ED127E0700000203F420F003C01002011
:108CE000601200207401002090130020CC1400209A
:108CF0002C0E00204C01002008160020B81E85EB29
:108D000051B8CE3F00000840A0860100983A00000C
:108D100000D02724640100207001002000040050CE
:108D2000E7030000624B4200D318069A12885A806B
:108D30008000604B5F4AD43B02905E4982189B8F53
:108D4000138030314118A26C4A605B4940185B497E
:108D500016300CC902F05CFB216EA06C884207DA69
:108D6000544A02995158012902D12066039905916C
:108D70005049029A8958814217DD012915DD2146A3
:108D8000002812DD0398C8840220087065730CE087
:108D90004B4A00210F2002F0D8FA6079E178401C9C
:108DA000814202D0002002F0E0F9208DA18D88429E
:108DB00000D248E6434A89188842FAD8A07B0128A5
:108DC00001D00220A07302F093F83D4A00210F2049
:108DD00002F0BBFA2179002917D03B4802889000A5
:108DE00013188B4200D22570002000F0E9F8A07C17
:108DF00000283BD02F496C310B78A3724878607201
:108E00008A782272022B17D030E0E16C226E323960
:108E100020468A420EDAC1792B4A491CC9B2C17177
:108E2000128852008A42E2D20599C184022101705F
:108E30006573DCE7E571DAE710280ED0C82815D293
:108E4000224BC91C1D60224B1818FCF797F903F040
:108E50004FF9642001F068FC31E61E4D286840009F
:108E6000000E03D1C878FCF710FC2860002023789E
:108E7000627B657910E00F4E0E4F4100303E183F87
:108E8000765A7F5ABE4205D00A4F0223002201269D
:108E9000483F7E52401CC0B2A842ECD3237062739C
:108EA000074A002180320F2002F04FFA09B0F0BDCE
:108EB000CC140020C013002060120020F00000201D
:108EC00000D02724983A00004C01002078010020AF
:108ED000EC0D002068010020F8B52E4C0546E06E30
:108EE0002D4A281A411E2067914215D21A21615E2F
:108EF000081AFCF7D1FB294A294BFCF7C5FA0646AC
:108F000032200F46205EFCF7C7FB32463B46FCF79B
:108F100009FAFCF7F7FB6086002060761D481C23E9
:108F2000C35E828C1F48008884461F4806881DE067
:108F30006046484380181D4F80B238803027784300
:108F40006427643078431A4F6066C01985420BD29B
:108F5000C8B2184932220880606EA25E411BC9184F
:108F60008918A166E066F8BD491C6176617EB14250
:108F7000DED33020424310486421101848430F4983
:108F80004118E16660663221401B615EC0184018DE
:108F9000A066F8BD70000020CF0700009A9999994B
:108FA0009999B93F5E0100204C0100207201002018
:108FB00078ECFFFF5C01002074270000C0BDF0FFCB
:108FC000FEB5294D2988491C8FB228492F800E886B
:108FD000FCF762FB264A274BFCF756FA01910090FA
:108FE00025483146FCF784F8244C218F4218B742BB
:108FF00006D3002028802248019E1018009D02E020
:109000001046019E009DFCF75BFB33462A46FCF7A9
:1090100089F9FCF79BFBA086012580B2ED03A842ED
:1090200001D3401BA086E08BFCF74AFB154A164B88
:10903000FCF792FA0646A08E0F460090FCF740FB24
:1090400032463B46FCF76EF9FCF780FB80B2E086C7
:10905000A84201D3401BE0860C490098096848618A
:1090600000982087FEBD00005C0100204C0100201C
:109070001904560E2D624040E17A00007000002075
:109080001F050000F853E3A59B843E40081600200E
:1090900070470000F0B589B0002004900A2002F06B
:1090A00095F87D20400102F0ABF8B34800228270B1
:1090B000C16BB34C491CC163B049C38D098A2546B5
:1090C000C918C1852146C2751331079147310391F3
:1090D0006D393135AB4F223005910290A64E0F21EC
:1090E000A948717100782071A84AB07912784000BF
:1090F0001043B27D92001043E071B08FE070000A1F
:109100002072A17431461E229C310798FCF736F874
:10911000402228469E49FCF731F8029903980A7BC1
:10912000C274497B0175092060729A480078A07268
:10913000B08C2073F07D410030469C3009180598B2
:109140000A78027549784175762000228C4902F030
:1091500027F970790621484300211C3002F032F9CA
:10916000022002F083F800210F2001F0AFFF384207
:109170003064F8D0306C411C18D040047ED5812278
:10918000D20100210F2002F0E0F80021102001F0B0
:109190009DFF41067A48490E0022B43001F0CCFF11
:1091A0007748B430417A022902D0BDE001F0DCF802
:1091B00002227949401DFCF705F80028F5D16E48D8
:1091C0000222C07D41006C489C3009186C48B530C3
:1091D000FBF7F8FF0028E8D102F045F9664AD167AD
:1091E000906702F02DF9644A803203C20498002887
:1091F0002CD1012004906248684E8C30C08E6049AA
:1092000030805D488C31098F41846548FDF72AFF25
:109210005949644A0885488CFF30C33080B248847D
:1092200090420CD952428018488430885D4A401CD4
:1092300080B20B323080904201D3002030803088E1
:109240007D22D20050434A8C801848654C486946BC
:109250008C30428E0A80808E488049490422B53184
:10926000C81FFF38FBF78AFF4348494AC07D009971
:10927000800011504049803103C900E075E0FF23B0
:109280005B040022C01851410906060A0E4330460D
:1092900001F095FF710849000A0E080236490026C0
:1092A0008031CA6088603448C36F826F3448483860
:1092B00002F0AEF8304880300CC83148443802F033
:1092C000A7F82D488030C36882682D48403802F0E6
:1092D0009FF82B49002252393C2002F061F800210E
:1092E0003C2002F06FF8012001F0C0FF2249087312
:1092F00008468078401C887001210520C9030007BA
:10930000FCF748FE1C48007B002805D100210F20F7
:1093100001F0DCFE0006F9D5802200210F2002F0CA
:1093200014F81548467002E01349012048701248AD
:10933000C17D491CC9B2C1750F2900D2CEE604987F
:10934000002810D10C4A1849908C002802D00B88B4
:10935000984201D908889084144980B20988401E37
:1093600048431349088009B0F0BD124A00210F207C
:1093700001F0EBFFD8E70000700000202C0E002069
:109380006012002000D027243C010020740100203E
:109390007C1400204C01002064010020700100209A
:1093A00008160020E70300004801002046010020C5
:1093B0004401002000902724F8B531492F48086067
:1093C00002F03AF92F4800F0A1F92F4CE0822D4825
:1093D000801C00F09BF920832A48001D00F096F9BC
:1093E00060832B4829494180014640310979294F42
:1093F0000906090E617006D1C7800121C1870A21C3
:10940000418700218187244AC18E1170C18F21714B
:10941000818F6171817AA17085880521A562618142
:10942000C6883046FBF764FEA08101462846FBF75C
:109430005FFE8800081885B2164825816843FCF74E
:109440003FF9164A164BFCF787F8FCF77FF9E081E5
:10945000658231463846FBF74BFE20820146C82024
:10946000FBF746FE608401202084FCF797FDA08274
:10947000E2890C490C48FDF7F9FDF8BD5DA1000833
:1094800068000020004F00083C0100202F0200006F
:10949000EC0D0020E803000018000020F853E3A5BD
:1094A0009B843E40FF7F000008160020F8B5744CF6
:1094B00000202071734D01202880734EC820308019
:1094C000E07A401CE072C00706D0A08C411EA18447
:1094D000022801D2C820A0840120C043FFF770FDFC
:1094E0000A2001F073FE7D20400101F089FE022177
:1094F0006648FDF789FB00287ED000206449800083
:109500000978654F49000843624909780843B872F1
:10951000102078726148C1887D20C000FBF7E8FD0B
:1095200078735F485D490078B87338460B308A78A5
:109530000270C97841705949421C20310B7ED370AA
:10954000497E11715549D01C22310B7E5371497EE1
:109550009171524940310A7C0271497C417100226B
:109560003946172001F01CFF0021172001F02AFFC7
:10957000022001F07BFE4B4F00210F2001F0A6FDE1
:1095800038422064F8D0206C411C77D0400471D55B
:109590008122D20100210F2001F0D7FE00211020EE
:1095A00001F094FD41063C48490E0022B430E165CB
:1095B00001F0C2FD384FB437787A11285AD102220F
:1095C0003949781DFBF7FEFD002853D1F81F027AB8
:1095D00069460A70407A4870B97A2980C820FBF73A
:1095E00087FD3080387BA0843846304D2838C08EC7
:1095F00028802348394600E03EE02839098F41841D
:109600002B48FDF72FFD2085608C2A49FF30C330A1
:1096100080B2608488420CD949424018608428880E
:109620002449401C80B20B312880884201D300209D
:10963000288028887D21C9004843618C40186065D6
:1096400000F0A4F868460088E0841349B87CC7316C
:109650006071420008460D466930FBF78FFD607966
:10966000294642001448FBF789FDA08CFF2801D051
:1096700003202070F8BD01E001203FE700F074FEF8
:10968000700000204C0100205E010020000400500A
:10969000400100204101002060120020EC0D00205C
:1096A0001800002000D02724640100207001002051
:1096B00008160020E7030000A813002070B586B04C
:1096C00014216846FBF773FD01250F4EED030022C0
:1096D00029463046FDF7A5FA0120002401900294A6
:1096E0006946009503943046FDF7D2F903200190B6
:1096F00002946946009503943046FDF7C9F90220AB
:1097000001F012F806B070BD0004005000887047E8
:1097100070470000F8B5044600206A461080194DD5
:1097200055222A70AA226A700322AA70661DEE7062
:109730002A716971144A49008918AC712246E81DE2
:10974000FBF71CFD002007E029186A46897812887B
:1097500089186A461180401CB042F5DB611DA81CC7
:10976000FCF77AFA01466846018029190078C87129
:1097700068464078087221460931024800F004FB2F
:10978000F8BD000046150020EC0D0020FEB5FFF7E7
:10979000A3FB2548FDF766FC244C86B2268560793C
:1097A0000A21081AC000FBF777FF07460191A06E57
:1097B000FBF786FF1E4A1F4BFBF7CEFE00900D46BF
:1097C0003046FBF77DFF2B46009AFBF7ABFD3A4690
:1097D000019BFBF7A7FDFBF7B9FF85B2A586E08BE0
:1097E000FBF76EFF124A134BFBF7B6FE06460F4619
:1097F0002846FBF765FF32463B46FBF793FDFBF738
:10980000A5FF81B20120C003E186814201D3091A7C
:10981000E186854201D3281AA0860349A08E0968F3
:1098200048612087FEBD000008160020700000205F
:10983000F853E3A59B843E40034A1168382389B25C
:1098400099430143116070470030014010B5FDF7A6
:10985000F5F910BD10B59AB034216846FBF7A7FCA6
:1098600014210DA8FBF7A3FC1C2112A8FBF79FFCF9
:109870001B4801680324E402A143C2148918016053
:10988000FDF76EFC17480169A143016106200090B5
:10989000FF2001300290012003901020049002204C
:1098A000099040040B90000100240C900A94684633
:1098B000FDF784FE0F200D9003200E900F9410945E
:1098C000012111940DA8FDF74FFD81201290032076
:1098D00080041890149412A8FDF794FC1AB010BDDF
:1098E000007000404010024010480168821511438A
:1098F0000160C1680E4A1140C16001680D4A114003
:109900000160816849084900816001680122920470
:1099100091430160C168FD2212049143C16000219E
:109920000161064904488860704700000010024049
:109930000C40FF88F6FFF6FE0050000800ED00E046
:10994000F8B5102405252D07AC62AF20800000F08B
:10995000F2FEAC6101F0CEFB2F4C304F304E606711
:109960000EE001F0C7FB6067FEF774FC606C411C01
:109970006164142804D92BA000F078FC2D48C7603E
:10998000606FB042EDD10026666420780127FF03A6
:10999000030000F0A4FC05040C192D303200012254
:1099A00039462846FDF73DF9FFF780FD06E0012224
:1099B00039462846FDF735F9FFF76CFB002239469A
:1099C0002846FDF72EF918E0607B0122401C6073E9
:1099D00039462846FDF725F9FCF7FCFA00223946FE
:1099E0002846FDF71EF9607B052806D9267004E09D
:1099F000FEF768FF01E0FFF74DFB02210E48FDF77F
:109A000003F9002805D000200C49087001F058FA2D
:109A1000F8BD0120F8E70000700000200400FA05FE
:109A20003001CADE4457204944204552524F522E3D
:109A30000D0A000000ED00E0000400507401002059
:109A400010B5818CC90707D001684A6801235B04FF
:109A50009A43836A1A434A60818C890707D5016853
:109A60004A6801231B049A43C36A1A434A60818CE3
:109A7000490707D501684A6801239B049A43036B91
:109A80001A434A60818C090707D501684A68012397
:109A9000DB039A43436B1A434A60818CC90607D59E
:109AA0000268916801231B039943836B19439160FA
:109AB000818C890607D501688A6801235B039A4374
:109AC000C36B1A438A60818C490612D503685A68B1
:109AD00001210905046C8A4322435A60026C8A42C0
:109AE00007D10268516803235B059943436C19430E
:109AF0005160818C090607D501684A680123DB049F
:109B0000806C9A4302434A6010BD0000F8B50446D9
:109B1000002680300660FDF78BF805462068006857
:109B2000124F000709D501212B4600224905204686
:109B3000009700F0A1FA00280DD1206800684007C6
:109B40000BD501212B46002289052046009700F005
:109B500093FA002801D00320F8BD2020A067E06719
:109B60002666603426750020F8BD0000FFFFFF0167
:109B7000F8B5154CC826E078002823D16079002874
:109B800020D101206071114D686B0027002818D08A
:109B9000686BC821081A0FE00D48E168405C6169F4
:109BA0008847E068401CE060E068C82800DBE760A8
:109BB000696BC820401A761EE168814201D0002EF0
:109BC000EADC6771F8BD000054000020000002408C
:109BD000240D002070B5224CE07800283FD1207978
:109BE00000283CD1012020711E4EF1690025090694
:109BF000002933DA2156625791420AD1F0694006B2
:109C00002CD5A079002829D0A5712089401C20815D
:109C100024E0A179002903D1A0710A2000F08BFD76
:109C200000202056CC2148430F49421820691218C1
:109C30001279B262401C00222061A256CC235A4302
:109C4000895881420ADC25612078401C20702078E8
:109C50000E2800D12570A078401CA070257170BD21
:109C60005400002000380140FC01002010B5806A3B
:109C70000022014640314A834A82FDF753FF10BD5E
:109C800070B5846AA06FE56F2168896800260906AF
:109C9000002906DA212804D152200653204600F07C
:109CA0006BF820688068400606D5222D04D15A2022
:109CB0000653204600F047F8204680300168102205
:109CC000114301602046FDF72DFF70BD10B5014620
:109CD0000968806A096889061CD400225A210A5240
:109CE00001680A68FF2301339A430A6001688A68A1
:109CF000520852008A6001688A6840239A438A6049
:109D00002021C167016E012904D101680A6810236E
:109D10009A430A60016E012902D0FEF7E5F810BDF2
:109D20005821095AFDF7FCFE10BD10B5806A016E7E
:109D3000012902D0FEF7D9F810BD5821095A490867
:109D4000FDF7EEFE10BD01680A68FF2321339A4338
:109D50000A6001688A68520852008A60016E01290F
:109D600004D101680A6810239A430A602021C16760
:109D7000002101664166704701680A68C0239A4362
:109D80000A6020218167704770B5164CE278002A7E
:109D90000CD12279002A09D10122E2700025C829BC
:109DA00003DC0222A256002A01DCE57070BD01230B
:109DB000E356CC2253430C4AD1500123E356CC2620
:109DC00073439B180A460146181DFBF7D7F96078C4
:109DD000401C607060780E2800D16570A078401E2D
:109DE000A070E2E754000020FC010020F8B5044612
:109DF000016880682369E669184363690025334375
:109E00001843724A0B68724E334003430B6021685B
:109E1000486803231B039843E3681843486021689C
:109E2000A069914201D0236A18438B680B26360241
:109E3000B34303438B606749236867488B420CD167
:109E4000C0688007800F06D0012839D0022835D09D
:109E5000032821D11EE001271FE060498B420AD16F
:109E6000C0680C21084027D0042829D0082825D014
:109E70000C2811D10EE093420ED1C168032080025C
:109E8000014019D001208002091A19D0091A15D0F1
:109E9000814201D1082700E010274F49504840393E
:109EA0008600934232D1002F0CD0022F0DD0042F08
:109EB00010D0082F7FD126E00027EEE70227ECE73D
:109EC0000427EAE7FDF71EFB06E00968C90605D48A
:109ED000304603E0FDF736FB002872D0626851007F
:109EE0005118814267D81103814264D3010E0602E2
:109EF0005008002330185941FBF710F903210902DB
:109F0000411A384A55E00120C003E7E70122E3691E
:109F1000D20393422BD13B0000F0E1F90906090C72
:109F20004D114D4D4D274D00FDF7ECFA09E0FDF7C1
:109F3000F9FA06E00968C90605D4304603E0FDF7E2
:109F400001FB00283DD0616840004A088018FBF7FB
:109F5000CFF880B20146244A103991422BD8511CC7
:109F600001400007400F084329E01046EBE73B00A3
:109F700000F0B5F90906090C211221212123210045
:109F8000FDF7C0FA0AE0FDF7CDFA07E00968C90657
:109F900006D4304604E00EE0FDF7D4FA002810D0D5
:109FA00061684A081018FBF7A3F880B201460E4A10
:109FB0001039914203D9012503E01046F0E72168EA
:109FC000C86000206066A0662846F8BD00480040D2
:109FD000F369FFEF003801404010024000440040A8
:109FE00000093D00FFFC0F00EFFF0000F8B504463C
:109FF0004165403000262746028380373E6022209C
:10A00000E0672546206F603500281CD01749C162E3
:10A01000216F17480863216F16484863206F8663D5
:10A02000236F606D9C4613462168024660462431CA
:10A03000FCF756FC002806D0102038602E75202032
:10A04000A0670120F8BD2E7520680168FF2201324B
:10A0500011430160206881680122114381602068FA
:10A0600081684022114381600020F8BDCD9C00082A
:10A070002B9D0008819C0008FFB581B005460F4666
:10A08000044660350A9E39E0701C37D0FCF7D0FDDD
:10A090000499401AB04222D8002E20D020680168CE
:10A0A00049072BD5C069C043000527D4012021688A
:10A0B000C002086220680168FF22A132914301605A
:10A0C000206881684908490081602020A067E06716
:10A0D0008034206000202875032005B0F0BD206882
:10A0E0000168FF22A132914301602068816849081C
:10A0F000490081602020A067E067EBE72068C16924
:10A100003846884305D0002103988142BCD0002006
:10A11000E3E70121F8E7000010B5044910200968C1
:10A1200008620248FDF700FD10BD0000D0160020B7
:10A1300001490D20887070475400002010B5FEF7CB
:10A14000BFFAFEF797FBC82202490348FDF79CFEC1
:10A1500010BD0000240D0020D0160020F8B53E4CA4
:10A16000002321783D4A1D46082910D0072947D0F1
:10A17000062950D0052952D0042953D0032954D0A0
:10A18000002956D0012958D002295AD05BE0A17885
:10A1900000264A1F04E0314FBF5DFB189BB2761CBE
:10A1A0009642F8DB667927799A195118E378627834
:10A1B000C9188918C9194018C0430006000E1AD1E1
:10A1C000012E14D0022E16D125482449C018FAF7C2
:10A1D000D5FF01F08DFF642000F0A6FABFF34F8F8A
:10A1E00021492048C860BFF34F8F00BFFDE75908E1
:10A1F0001046FFF78FFA2570E570A570A571F8BDC0
:10A20000A1795054491CC8B2A071A178491F884255
:10A21000F5D1082001E0607007202070F8BDE070E3
:10A220000620FAE760710520F7E7A070E5700420CA
:10A23000F3E7552807D10120EFE7AA2803D1022030
:10A24000EBE7032803D02570E570A570F8BD032067
:10A2500020702071F8BD000034010020E2140020BD
:10A26000EC0D00200400FA0500ED00E010B5024AF4
:10A27000024900F0E5F910BD29B400088C01002066
:10A280002021020C01D010211046020A01D01046F4
:10A290000839020901D01046091F820801D0104672
:10A2A000891E420801D0881E7047081A7047F8B509
:10A2B000040C8BB2264682B25E430D0C1046370C5E
:10A2C0005843360480190021794116466E43370CF5
:10A2D00036048019794126466E438919F8BD30B499
:10A2E0007446641E2578641CAB4200D21D46635D33
:10A2F0005B00E31830BC18474900CA020243100053
:10A3000000D004204A0D01D001221043044A490D17
:10A31000914201D102210843012800D10520704754
:10A32000FF0700008307FF22DB0E9A408907090E12
:10A330009940002808DB830809489B001B1818680F
:10A3400090430843186070470007000F08388308DF
:10A3500004489B001B18D86990430843D861704794
:10A3600000E400E000ED00E0BFF34F8F0449034834
:10A37000C860BFF34F8F00BFFDE700000400FA057F
:10A3800000ED00E0F8B504464F1EC800083821185B
:10A3900015461E46086849683A4606239A4310D077
:10A3A0002A463346FBF770F83A46D200083AA3181B
:10A3B0001A687F1E5B68FAF7B5FF06223B46934397
:10A3C000EED1022F23D0042F11D0062F2FD12A46F1
:10A3D0003346FBF759F8E36AA26AFAF7A3FF2A4665
:10A3E0003346FBF751F8636A226AFAF79BFF2A4665
:10A3F0003346FBF749F8E369A269FAF793FF2A4667
:10A400003346FBF741F863692269FAF78BFF2A4666
:10A410003346FBF739F8E368A268FAF783FF2A4668
:10A420003346FBF731F863682268FAF77BFFF8BD23
:10A43000002210B5134610460149FBF78DF810BDF8
:10A440000000F03F10B5FAF76DFF10BD002210B507
:10A45000134610461146FBF77FF810BD10B50721D3
:10A46000024A00200907FBF7EFF810BD01030000C6
:10A47000034A10B500201107FBF7E6F810BD0000F5
:10A4800001FDFFFF02E008C8121F08C1002AFAD12F
:10A4900070477047002001E001C1121F002AFBD164
:10A4A00070470000014908607047000090010020DB
:10A4B00008B50021684601706B46012202212C205C
:10A4C00000F052FF0221684601706B4601222C20E9
:10A4D00000F04AFF08BD000038B504466D2069460B
:10A4E00008706B46012207492E2000F03DFF064907
:10A4F000002C01D0054A00E0054A2E2000F01AFF8A
:10A5000038BD00000608000006180000070600001D
:10A510000716000038B504466B460222002136209B
:10A5200000F0EEFDB3212300FFF7D9FE0E0F081552
:10A530003A3A3A3A1C273A3A2F34483A00216846C8
:10A54000017040784108490014E0694608788008A5
:10A550008000401C04E06946087880088000801C68
:10A5600008701DE0684602780A404832027041785F
:10A57000802001436846417012E0684602780A4034
:10A58000027040784106490EF4E769464878022196
:10A59000084303E069464878FD2108406946487051
:10A5A0006B4601220021362000F0DEFE012200ABC6
:10A5B00011463620013300F0D7FE38BD69460878D1
:10A5C000CF21084069462030CAE708B50321684614
:10A5D0004170012101706B4602220021362000F0FB
:10A5E000C3FE0122D20306212D2000F0A3FE01208C
:10A5F00000F09AF80120FFF78DFF08BD08B5020AA8
:10A6000069464A7008706B46022204212D2000F032
:10A61000ABFE0320694608706B46012206212D20FF
:10A6200000F0A2FE0020694608706B460122062158
:10A630002D2000F099FE0A212D2000F047FD08BDD5
:10A64000F8B516460F460446002503E03946B047E4
:10A65000641C6D1C20780028F8D12846F8BD000045
:10A66000F8B54A002B4B520DD6182B4A0C4605461E
:10A67000142E2BDA002E12DA284BFAF753FE0022A2
:10A680001346FBF7A9F840D2002C03DA0124E407B3
:10A6900000253AE02046284337D0214C14E0214FD2
:10A6A0000B46F7403B402B4331D01C4BFAF73AFEA8
:10A6B00000221346FBF790F827D2002C03DD01207F
:10A6C0000005F0400419BC4300251EE0332E1EDCBB
:10A6D00033460027143BFF43DF40384217D00F4B6F
:10A6E000FAF7CAFE00221346FBF776F80DD2002CCB
:10A6F0000ADD142E0CD03420811B01208840401923
:10A70000A84200D2641C0546BD4321462846F8BD38
:10A71000641CF9E701FCFFFF9C7500883CE4377E70
:10A720000000F03FFFFF0F007D2110B5C900484336
:10A7300000F001F810BD002140E000BF00BF00BFE5
:10A7400000BF00BF00BF00BF00BF00BF00BF00BF11
:10A7500000BF00BF00BF00BF00BF00BF00BF00BF01
:10A7600000BF00BF00BF00BF00BF00BF00BF00BFF1
:10A7700000BF00BF00BF00BF00BF00BF00BF00BFE1
:10A7800000BF00BF00BF00BF00BF00BF00BF00BFD1
:10A7900000BF00BF00BF00BF00BF00BF00BF00BFC1
:10A7A00000BF00BF00BF00BF00BF00BF00BF00BFB1
:10A7B00000BF00BF00BF00BF00BF491C8142BCD327
:10A7C0007047FFB581B01E460F46040026D00B9996
:10A7D00003980143A06A3943826807209047002804
:10A7E00018DB0A99A06A3143826806209047002846
:10A7F00010DB25462035A979032F01D90820014314
:10A80000032E01D904200143A06A826809209047E1
:10A81000002806DA0120C04305B0F0BD0020C04387
:10A82000FAE7384600F000F92060304600F0FCF806
:10A8300060600A9868700398A870EF702E710B988A
:10A8400068710020E8E70000F7B50446002090B0EA
:10A8500000900190002C05D06A46062101F082FC90
:10A86000062803DA0020C04313B0F0BD68464078E4
:10A8700001026846007800040918684680780818C4
:10A88000FAF71EFF05466846039100790102684603
:10A89000C07800040918684640790818FAF710FFD4
:10A8A000032206460F4692075C4BFAF795FF07D244
:10A8B00000225B4B30463946FAF7D8FD06460F4674
:10A8C00003229207554B28460399FAF785FF07D2D2
:10A8D0000022534B28460399FAF7C8FD0546039119
:10A8E0002068FAF7EDFE02460B4630463946FAF785
:10A8F00033FE07460A200791205EFAF7CDFE3A465E
:10A90000079BFAF7C1FD064608200991205EFAF779
:10A91000B1FE0021C943FAF7F9FCFAF735FF3246D8
:10A92000099BFAF7FFFC069108906068FAF7C8FEE9
:10A9300002460B4628460399FAF70EFE05461A20F2
:10A940000E46205EFAF7A8FE2A463346FAF79CFD2B
:10A950000C9009911620205EFAF79EFE099B0C9A36
:10A96000FAF7E0FC05910A902A46334638460799E3
:10A97000FAF78AFD059B0A9AFAF786FD05910A9077
:10A980001420205EFAF788FE3A46079BFAF77CFD12
:10A9900007461C200791205EFAF77EFE2A463346C2
:10A9A000FAF772FD0E900B911820205EFAF774FEF4
:10A9B0000B9B0E9AFAF7B6FC2A463346FAF764FD6B
:10A9C0000B910E902069FAF767FE0B9B0E9AFAF72F
:10A9D000A9FC2A463346FAF757FD05460E46E068BD
:10A9E000FAF75AFE2A463346FAF79CFC3A46079B8A
:10A9F000FAF798FC059B0A9AFAF794FC0122920751
:10AA0000084BFAF741FD02460B46129C089806993E
:10AA100003C411980CC0002026E70000FFFF5F412F
:10AA200000007041E17A843F00B50121C9040300B0
:10AA3000FFF755FC081A05080B0E1114171A03200E
:10AA4000C00400BD0720C00400BD0F20C00400BD2D
:10AA50001F20400300BD3F20400300BD7F20400376
:10AA600000BDFF20400300BD084600BDFEB5264FD7
:10AA70000D4604000FD0002D0DD0264600202036B4
:10AA8000B071F07129680D208847002801DA78003C
:10AA9000FEBD102801D03846FEBDA562E968002938
:10AAA00001D028208847204600F030F80028F3DB4A
:10AAB000A06AA52182680E209047A06A962182682C
:10AAC0000F209047A06A0221826862209047A06A06
:10AAD000002182680E209047A06A002182680F2022
:10AAE00090477179302001910090062320220121A6
:10AAF0002046FFF766FE0028CEDB204600F0AEF8C9
:10AB00000028C9DB0020FEBDFFFFFFFF10B586B0A7
:10AB1000044614216846FAF74AFB002C7ED0A06A4E
:10AB2000122143686A4610209847122877D1684658
:10AB300000780122010168464078120300090818D4
:10AB400043492081884201DD801A2081684683784C
:10AB500040780007000D18186081884201DD801AD6
:10AB6000608168460079012201016846C0781205BB
:10AB70000003091868464079000908183549E06063
:10AB8000884201DD801AE060684640790007030BC7
:10AB90006846807900021B186846C0791818206141
:10ABA000884201DD801A20616846417A007A0002FD
:10ABB000081802B2284801210904A282824201DD5C
:10ABC000521AA2826A46D37A927A12029A1812B262
:10ABD000E282824201DD521AE2826A46537B127B94
:10ABE00012029A1812B22283824201DD521A228383
:10ABF0006A46D37B927B12029A1812B26283824217
:10AC000001DD521A62836A46537C127C12029A1842
:10AC100012B2A283824204DD501A01E00BE008E088
:10AC2000A083A06A016828208847002806DA01204E
:10AC3000C04306B010BD0020C043FAE7C011C007F2
:10AC40002034002800D0802060710020F1E700004F
:10AC5000FF070000FFFF0700FF7F000010B50400A2
:10AC600009D0A06A0721826808209047002805DAE9
:10AC70000120C04310BD0020C04310BD0720203478
:10AC80002070002010BD0000FEB504460020019099
:10AC900000906079734940000E5A61782578491E0A
:10ACA0007148CFB20163042D77D0072D75D00021F4
:10ACB0000291217801736C49E37901229205896937
:10ACC000002B6CD0914381616748217A4173217ACE
:10ACD00082698907890B0A4382610021042000F000
:10ACE00034FB324661492E2000F024FB3846FFF742
:10ACF000F3FB5F4E0522705D810040185D494318EB
:10AD000007212B2000F030FB5B49029801220B1831
:10AD10000B21282000F028FB705D584980000A585C
:10AD20000C21282000F011FBE079554980004018E3
:10AD3000A1794900425A0221272000F0FBFA51482C
:10AD40007E00825B0421272000F0F4FAE0790028DD
:10AD500029D0A07804282CD0282069460872202207
:10AD60000621272000F0E6FA02AB01222621272047
:10AD700000F0FAFA444938014018E1788900425855
:10AD80000821272000F0E1FAA17A601C627A09020A
:10AD9000114313D016E000E001E0012188E71143E0
:10ADA000F608816190E764220621272000F0C2FAAC
:10ADB000E0E71020694608720246D1E73349017284
:10ADC000090A4172417A007A0A02024320212720AF
:10ADD00000F0B0FA2E4F0C2123203A6800F0B5FAAB
:10ADE000F01982880421232000F0A4FAA079002819
:10ADF0000BD0E0792749012243180021212000F0DF
:10AE0000B3FA03200190012000902A07120F1001CD
:10AE10000243607800218007000B0243019800057F
:10AE200002430098400402432079C00640090243CF
:10AE30006079C00602431F2000F087FAA07861788D
:10AE40000123084302040848DB030261E179490356
:10AE500019430A4302610021082000F076FA00201D
:10AE6000FEBD000098C20008C001002004280000B8
:10AE700040C20008240000204200002048C2000810
:10AE800068C2000874C2000878C2000841100000BF
:10AE900060C200084400002038B50C4607498A8B80
:10AEA000002102432C2000F045FA684604706B46EE
:10AEB000012206212C2000F057FA38BDC0010020E5
:10AEC00010B5FFF7F5FA10BD10B504460421362081
:10AED00000F0FCF80121C902002C01D0084300E079
:10AEE000884302460421362000F02FFA10BD0000EE
:10AEF00038B540206946087000210E2000F0E6F8C1
:10AF00000446002211460E2000F01FFA6B46012273
:10AF100000210D2000F028FA074A00210F2000F040
:10AF200014FA00F0EDF9224600210E2000F00DFA8F
:10AF300002480021017338BDF8FF2724E0010020FA
:10AF4000FEB50546042069460870514C0020607526
:10AF500021462031206348710873A0836063A06399
:10AF600000F0C8F84B4E206002E000F0C3F820600B
:10AF7000B042FAD10020FFF7CDFA00F0BBF8464E00
:10AF800020603078242801D9243806E00621FAF719
:10AF9000AFF80622101A40010843020601040A43D2
:10AFA00001020A430243B260706000211E2000F0DB
:10AFB000CCF900F09FF820606B460122002124208C
:10AFC00000F0D2F91E20FFF719FB86B2300AA073F9
:10AFD0000420FFF713FB074600F08CF820603806CA
:10AFE000000E0DD002206946087101AB012212212A
:10AFF0002D2000F0B9F9A08B012109030843A0839B
:10B0000000F078F820600620FFF7F8FA606007206B
:10B01000FFF7F4FAA060F006C00E207501D11020F1
:10B020002075C0B200F0DCF9E80707D0FFF7CDFAD1
:10B03000A08B0121C9020843A0830AE00521362024
:10B0400000F02EF81549084002460521362000F090
:10B0500071F90120FFF75EFA0021042000F036F8B4
:10B06000A0610021262000F031F815218903084352
:10B0700002460021262000F068F900222621362011
:10B0800000F058F900F036F820600020FEBD000006
:10B09000C00100203001CADE18000020FFFD0000C2
:10B0A00038B5094C89B280B26B46022200F028F80C
:10B0B000002806D1684640780102684600780818E2
:10B0C00084B2204638BD0000FFFF000038B50024E0
:10B0D000E44389B280B26B46042200F011F80028E4
:10B0E00006D103216846435C2202D418491EFAD5D2
:10B0F000204638BD10B500210846FFF7E7FF10BD18
:10B1000038B5002909D0402420436C462070C8B2CD
:10B110007F2906D8607002200AE069460870012085
:10B1200006E0802420436C466070C809A0700320AC
:10B13000694600F0B7FF38BD10B5144603460A460D
:10B1400021461120FFF7DCFF10BD10B50346052294
:10B1500000211520FFF7D4FF10BD10B503460522CE
:10B1600000211720FFF7CCFF10BD38B505460020A1
:10B170006946087000F0C4F8FF2401342246002D0F
:10B1800001D00322120200210D2000F0D3F8002D7F
:10B1900013D06B46012203210F20FFF7B1FF684651
:10B1A0000078000709D5FFF7A3FE224600210D20F5
:10B1B00000F0C0F80020C04338BD002038BD10B5F5
:10B1C000024601210A2000F0C0F810BD10B5044667
:10B1D00000211A20FFF77AFF000D22030005120B51
:10B1E000024300211A2000F0B0F810BD10B502464D
:10B1F00002492E2000F09EF810BD00000418000047
:10B20000F8B505466B46012203210420FFF778FFBD
:10B210000126114C3607002D0DD02A4600210C20A6
:10B2200000F088F8694608781021084369460870DC
:10B23000A069304307E069460878EF210840694675
:10B240000870A069B0430B46A061012203210420CD
:10B2500000F08AF8F8BD0000C001002010B50246D9
:10B260000021182000F066F810BD0000F8B5074670
:10B27000002568460570B807204C2E4600280ADADB
:10B280008020694608706B46012200210D2000F0E5
:10B290006BF801202073F8076946087821D0062151
:10B2A0000843694608706B46012200210D2000F01A
:10B2B0005BF803210F20FFF7F3FE8121C90008424C
:10B2C00019D04020694608706B46012200210D20EC
:10B2D00000F04AF80020FFF7F7FD00252673ED4344
:10B2E00009E002210843694608706B4601220021EB
:10B2F0000D2000F039F82846F8BD0000E0010020DC
:10B300001CB56B46012203210F20FFF7F9FE6846AA
:10B3100000784022C1091040C9014000814208D094
:10B32000012069460871024601AB03210D2000F09F
:10B330001BF81CBD08B56B461A70120A5A7089B208
:10B3400080B2022200F010F808BD38B500236C4628
:10B35000E254120A5B1C042BFADB89B280B223464A
:10B36000042200F001F838BD38B58024002909D046
:10B37000C02528436D462870C8B27F2907D8687059
:10B38000022009E0204369460870012004E02043C0
:10B390006870C809A8700320694600F02DFF38BD09
:10B3A00010B51446012312189B029A4202D90020BC
:10B3B000C04310BD0B46821E21460920FFF7D4FF73
:10B3C000002010BD10B5054A8905126901430A43E2
:10B3D00000210820FFF7B9FF002010BDC0010020A8
:10B3E00038B504466B4601220E212B20FFF788FE5C
:10B3F00068460078E10640094001C90E01436846ED
:10B4000001706B4601220E212B20FFF7ADFF38BDE6
:10B4100010B5002142541C06120A22431B0A491C83
:10B420000429F7DB10BD000013B501231A46694655
:10B430000248FCF75BFD00981CBD0000D016002000
:10B440007CB5002425466846FFF77FFE0420694648
:10B45000220E2D02154322020C5C1443401EF7D528
:10B46000204629467CBD7CB5002425466846FFF76A
:10B4700074FE04206946220E2D02154322020C5C44
:10B480001443401EF7D5204629467CBDFBF7DEFB62
:10B49000FEF7E0F9FDF728F940494148002522C0B0
:10B4A00005608561C5613F490562C1600838FBF7E9
:10B4B00063FDFDF705F9FDF7DDF9FDF7B9F9FDF7D6
:10B4C000CBF8052401222407D1032046FBF7A9FB72
:10B4D000FDF772FFFCF7A8FFFAF760FBFAF71CFC18
:10B4E000FAF7EAFBFCF784FD0721A015FFF7D4FC6F
:10B4F000FFF7E6FC012211032046FBF792FB2848E8
:10B50000C8222949C830FCF7BFFCFCF73BFF274F96
:10B51000274E284C387800280ED13078002801D0EA
:10B52000032809D140212448FBF76EFB002803D1F2
:10B5300001210846FBF734FEE07800282AD0607825
:10B54000002827D0E57072B620780F280AD901208C
:10B55000194900038861FEF7F3F901201649000339
:10B5600088620CE0012251031348FBF75AFBFEF7F7
:10B57000E7F90121002249030F48FBF752FB62B6AD
:10B58000FCF768FEFAF72EFBA08C0028C2D0401E04
:10B59000A084BFE7FCF75EFEBCE70000007C004033
:10B5A00008160020FFFF0000240D00205A00002094
:10B5B000840000203C0100200004005010B586B03B
:10B5C000FCF7E0FE1748FBF75AFC14216846F9F730
:10B5D000EEFD154800900320019000200290052008
:10B5E00069460007FBF754FA69461048FBF750FA22
:10B5F00069460F48FBF74CFA01210846FBF7D0FDDE
:10B60000FF2401342046FBF7A3FD0A490868042201
:10B61000104308602046FBF7ABFDFBF7B1FD06B019
:10B6200010BD000008160020FFFF000000040050BD
:10B63000000800500070004010B501229202164927
:10B640001648FAF7EDFB1448154902888A4222D0C1
:10B65000018014498180FF21F531C1800A210181D7
:10B6600000211E224181D24382810122C281818335
:10B670004323C3860287782343878287C287024693
:10B680004032118451849184C18391801423838238
:10B69000118200F02DFD10BDEC0D002000FC000813
:10B6A000AA55000034120000F0B51FB496B08446CD
:10B6B0000C460246199D18980390490068006300E3
:10B6C000490840080193002A01D0012600E0002625
:10B6D0009E19FE4BF6185B109E422BD36E00039F03
:10B6E0000296002F00D00127F719F84EF84BBE192B
:10B6F0009E421FD3039E0346F64F334309D03B4679
:10B700009C4201D1002A04D0019B002A05D00126C9
:10B7100004E0002039461BB0F0BD00269E19EE4B18
:10B720009E4207D8039F029E002F00D00127F619E2
:10B730009E4207D92B4660462146189AFEF782FEA4
:10B740001BB0F0BD0023002C29DAE44EB04226DA0B
:10B75000E34EB04201DB022321E0DE4EB0421EDBAD
:10B76000E04E070DBE19142E09DD3427BF1B039EC2
:10B77000FE400196BE40039FBE420BD00FE0039FE8
:10B78000002F0CD11427BF1B0646FE400196BE4079
:10B79000864204D1019BDE07F60F02239B1B0E4657
:10B7A000164318D1002D16DA002C03D0022B01D03D
:10B7B000012B06D00220FEF775FEFEF739FE1BB006
:10B7C000F0BD0220FEF76EFEFEF732FE0122D20728
:10B7D00051401BB0F0BD039E002E61D1BF4EB04260
:10B7E00020D1C148844201D1002A08D0B948814201
:10B7F00009DB002D10DB189829461BB0F0BD002096
:10B80000B4491BB0F0BD002D06DA01222946D2074B
:10B81000189851401BB0F0BDB44979440868496894
:10B820001BB0F0BDAB4FB84225D1002D1FDA002967
:10B8300004D0B14212D1002A09D018E0002A72D1F6
:10B84000A649E20F0020D20711431BB0F0BD002033
:10B85000E20F0146D20711431BB0F0BDB14206DA38
:10B86000234600203946F9F777FE1BB0F0BD10469D
:10B8700021461BB0F0BDB14212DA0126B607B5422F
:10B8800003D1234610461946FEE3994EB54207D12F
:10B89000261E05DB1046314600F040FC1BB0F0BD13
:10B8A00067007F081646002A40D100290AD08B4A3B
:10B8B000914229D1002C0EDD002D1CDB0020114609
:10B8C0001BB0F0BD022B16D0002C14D0012B12D1CE
:10B8D000002C14DB0FE0002C28DA002D09DB012BF3
:10B8E00003D000207D491BB0F0BD002081491BB072
:10B8F000F0BD012B03D0002001461BB0F0BD00209D
:10B900000121C9071BB0F0BD724A91420ED1002C33
:10B9100001DA002B17D0022B06D00020C043F9F724
:10B92000BBFE1BB0F0BD90E20120F8E7E217521C0D
:10B9300094461A4307D000220892664C62465B1E6A
:10B940001A4307D009E00120FEF7ACFDFEF77EFDAB
:10B950001BB0F0BD0022644C0892674A90427DDD26
:10B96000664B674A98421FDD914202DC002D05DBE1
:10B970004DE05848814217DB002D48DD0220FEF7DC
:10B9800091FDFEF76BFD05460E460022534B214606
:10B990000898F9F779FD084671004908C00FC007FB
:10B9A000014328461BB0F0BD914215DA002D2EDA76
:10B9B0000220FEF777FDFEF751FD05460E460022F8
:10B9C000464B21460898F9F75FFD72005208C80FF0
:10B9D000C0070243114617E03E4B994223DD002D7C
:10B9E00015DD0220FEF75EFDFEF738FD05460E462A
:10B9F00000223A4B21460898F9F746FD08467100A7
:10BA00004908C00FC007014328461BB0F0BD022003
:10BA1000FEF748FDFEF72CFD49004908E20FD2076A
:10BA200011431BB0F0BD002230463946F9F71EFD28
:10BA3000012205460E46D243F9F706FE314A324B43
:10BA4000F9F71AFD2A463346F9F71EFD0022284B66
:10BA5000F9F712FD07462A46334600E064E00391F9
:10BA600010461946F9F710FD3A46039BF9F70CFD0D
:10BA70000746032209915207244B28463146F9F71D
:10BA800003FD07910C90224A204B38460999F9F79B
:10BA9000FBFC074601911F4A1F4B28463146F9F728
:10BAA000F3FC3A46019BF9F7E1FC07460B460246D8
:10BAB000099107990C98F9F735FC00250E462846A0
:10BAC000079B0C9AF9F7D2FC3A4627E0FFFF1F00CC
:10BAD000FFFF0F000000F03F0000E0FF0000F07FDC
:10BAE0000000404301FCFFFF0000F0BF5A0B0000C4
:10BAF0000000E03F0000F0FF0000E0410000F043E4
:10BB0000FFFFEF3F555555555555D53F4715F73F65
:10BB1000FE822B6544DF5DF80BAE543E099BF9F7BE
:10BB2000ABFC02460B4652E1012500202D05A9423F
:10BB300007DA352230463946F9F786FD06463420C5
:10BB4000C0430A151218FE48101803900803FD4957
:10BB5000000B01430F46FC49884201DC002003E052
:10BB6000FA49884202DA0120119005E00020119084
:10BB70000398401C7F1B039011980597C200F4485E
:10BB80000F927844801843680268394630460D9316
:10BB90000292F9F76BFC07910C9030460D9B029ACC
:10BBA0000599F9F7BFFB02460B460020E549F9F776
:10BBB000D3FC09910490079B0C9AF9F765FC12904D
:10BBC00000201090E3480D46784400680E90012153
:10BBD00078104907084311990D9B890440180121E9
:10BBE000C90447183946029A0E98F9F73FFC3246C5
:10BBF000059BF9F741FC02460B4629461098F9F7D8
:10BC000043FC064602913B4629460E9A1098F9F7E6
:10BC10003BFC079B0C9AF9F72FFC3246029BF9F785
:10BC200025FC099B049AF9F72FFC0591129A0A90BA
:10BC30002B4610461946F9F727FC06460246C64829
:10BC40000F460B4606217844FEF79CFB32463B46E6
:10BC50000091049010461946F9F716FC009B049ACF
:10BC6000F9F712FC06460F462B461946129A109811
:10BC7000F9F758FB059B0A9AF9F706FC32463B4652
:10BC8000F9F750FB109A079104902B46104619467D
:10BC9000F9F7FAFBB14E0022334609910290F9F709
:10BCA00041FB079B049AF9F73DFB0020074602463B
:10BCB00033460091F9F7DAFB099B029AF9F7D6FBB4
:10BCC000079B049AF9F7D8FB06460D913A46294698
:10BCD000009B1098F9F7D8FB07910C902B46304643
:10BCE000129A0D99F9F7D0FB05460E463A46009B8D
:10BCF00005990A98F9F7C8FB33462A46F9F712FB6B
:10BD000002460B460746099107990C98F9F70AFB7A
:10BD100000250E462846079B0C9AF9F7A7FB3A46E2
:10BD2000099BF9F7A9FB07460722099152078C4B9B
:10BD300031462846F9F7A8FB07910090894A884BBD
:10BD400038460999F9F7A0FB07460191864A874BC7
:10BD500031462846F9F798FB3A46019BF9F7E2FA93
:10BD6000834B7B440F9A9B181A685B68F9F7DAFAE1
:10BD7000029009910398F9F78FFC05910490099BB3
:10BD8000029A07990098F9F7CDFA7A4B7B440F9AFB
:10BD90009B181A685B6817460393F9F7C3FA059B6B
:10BDA000049AF9F7BFFA0E462846059B049AF9F75C
:10BDB0005DFB3A46039BF9F759FB079B009AF9F79D
:10BDC00055FB099B029AF9F757FB02460B46199956
:10BDD00000200C900F461898F9F756FB029104903A
:10BDE0003B460C9A19991898F9F740FB2A463346B6
:10BDF000F9F74AFB029B049AF9F794FA09910E901D
:10BE00002A46334639460C98F9F73EFB06460F465C
:10BE1000099B0E9AF9F786FA574A0D46914220DBA4
:10BE20005242AA18024310D132463B46F9F71EFB94
:10BE300004900391514A524B09990E98F9F772FAFE
:10BE4000039B049AF9F7C8FC1ED20220FEF72AFBD6
:10BE5000FEF704FB49004908E20FD20711431BB06B
:10BE6000F0BD6A00474B52089A420DD3464AAA18C1
:10BE7000024300D0CBE532463B46F9F7F7FA099B7F
:10BE80000E9AF9F7A9FCF5D96800002340082C495F
:10BE90000393020D3D4B5218984223DD012000050B
:10BEA000521CD04042195000400D40183849794486
:10BEB000096813468C463749C1408B431203012160
:10BEC000120B090551181422101AC1400391002DBC
:10BED00001DA48420390624630463946F9F7C6FA1D
:10BEE00006460F4632463B4609990E98F9F71AFA6C
:10BEF00000252A46284B28460591F9F7C5FA0791EF
:10BF00000C90264A264B28460599F9F7BDFA009170
:10BF1000029032463B4628460599F9F7A7FA099B55
:10BF20000E9AF9F7A9FA1F4A1F4BF9F7ADFA009BD1
:10BF3000029AF9F7F7F907460B460246099135E0F0
:10BF400001FCFFFF0000F03F8E9803007AB60B0063
:10BF50006A070000AC070000D60600000000084099
:10BF600009C7EE3FFD033ADCF5015B14E02F3EBE4E
:10BF7000AA0500007005000000009040FE822B65BD
:10BF80004715973C00CC904000346F3F0000E03FE5
:10BF9000C6040000FFFF0F00432EE63F396CA80CDB
:10BFA000615C20BEEF39FAFE422EE63F07990C98FD
:10BFB000F9F7B8F905460E46079B0C9AF9F756FAB9
:10BFC0003A46099BF9F758FA09912A4633460E90EA
:10BFD00010461946F9F758FA074602462F480B460D
:10BFE000059105217844FEF7CDF93A46059BF9F70E
:10BFF0004BFA2A463346F9F73FFA0746019128469D
:10C000003146099B0E9AF9F73FFA099B0E9AF9F708
:10C0100089F9012304910C9000229B07384601996D
:10C02000F9F724FA05910E903A4628463146019BCD
:10C03000F9F72AFA059B0E9AF9F78EFA049B0C9AE7
:10C04000F9F714FA2A463346F9F710FA0022144B8E
:10C05000F9F712FA064603980D460005411909152D
:10C06000002912DC30462946039AF9F7EDFAFEF76B
:10C0700043F9042801D1FEF7FBF930462946039A1B
:10C08000F9F7E2FA064601E004E029180B463246C9
:10C0900021460898F9F7F8F91BB0F0BD68030000D5
:10C0A0000000F03FF0B58C46002510260521090759
:10C0B0008E620E4C08E067467F5DE760A768FF0769
:10C0C000FCD0E7681F706D1C8542F4DB002007463A
:10C0D00006E0E760A568ED07FCD0E5681D54401C4C
:10C0E0009042F6D38E610020F0BD00000030014088
:10C0F00070B572B60124074DA40221462846F9F70F
:10C1000075FE002804D0224603492846F9F712FF9D
:10C1100062B670BD00FC0008EC0D0020F8B50646C4
:10C120000C46F9F767FC051E0F4600D001200143BD
:10C1300049000B484908411AC90F0DD0002E01D003
:10C14000012100E000210C4361004908401AC00FA2
:10C1500002D10120FEF7A6F928463946F8BD0000B5
:10C160000000F07FF8B515460E460746002407E0AC
:10C170003819C0B200F008F8641C2870E4B26D1CD5
:10C18000B442F5D33046F8BD10B50446FBF7F6FFD0
:10C19000EE20FBF7C3FFFCF731F82046FBF7BEFFAC
:10C1A000FCF72CF8FBF7EAFFEF20FBF7B7FFFCF7F3
:10C1B00025F80020FBF782FF0446FBF7FDFF204631
:10C1C00010BD704770B50D460446FBF7D7FFEE2053
:10C1D000FBF7A4FFFCF712F82046FBF79FFFFCF7E4
:10C1E0000DF82846FBF79AFFFCF708F8FBF7E4FF89
:10C1F0000A20FEF7A0FA70BDF0B50025102605272D
:10C200009C463F070B46BE620C4C06E0595DE16060
:10C21000A168C907FCD0E1686D1C8542F6DB0020EF
:10C2200007E06146095CE160A168C907FCD0E168EC
:10C23000401C9042F5D3BE610020F0BD00300140AB
:10C240000000010203040005405C0000A05C040043
:10C25000C06C0800805C0400E03F1E00E07D1E0012
:10C2600007A9022570889B880A00160001000600B5
:10C270000100020087008D002D001A3152001A3390
:10C280009A001A351D011A376B003B31BE003B3353
:10C290005E013B3596023B37000099599959EB51A5
:10C2A0008F421E45142E0080EB51F5283333E13ABE
:10C2B000703DE13AC235852BC2353333C235C235C4
:10C2C000AE47E13A5138A330513800000000000079
:10C2D00000000102030406070809030406080C1005
:10C2E00018203000000000010203040000000000DC
:10C2F000000000000000F03F000000000000F83FD8
:10C3000000000000000000000000004003B8E23F11
:10C31000000000000000000006D0CF43EBFD4C3EC3
:10C32000033333333333E33FFFAB6FDBB66DDB3FB8
:10C330004D268F515555D53F01411DA96074D13F00
:10C3400065DBC9934A86CD3FEF4E454A287ECA3FFA
:10C350003E5555555555C53F93BDBE166CC166BF7C
:10C360002CDE25AF6A56113FF16BD2C541BDBBBE75
:10C37000D0A4BE726937663E0000000000000000D5
:10C38000A0C300080000002094010000BC5A00086F
:10C3900004C40008940100206C1A000094A4000852
:10C3A0000124130704380D091E080540082609104A
:10C3B0004008560A131D043B08BE0516D8BC4010A1
:10C3C000085201033AC842077052030CE5800C1B67
:10C3D0000202DD140901022281F01F66810498899E
:10C3E000968696798215980398149887967497780C
:10C3F00082439788967197778249F1013D2943924C
:04C400000492200082
:04000005080050C1DE
:00000001FF
